:020000040800F2
:100000000007002011020008B92C0008712C00081C
:10001000992C0008712C0008912C0008130200088C
:10002000130200081302000813020008AD3C000888
:10003000130200081302000813020008130200084C
:10004000130200081302000813020008130200083C
:10005000130200081302000881630008A963000866
:10006000D1630008F9630008216400081302000846
:10007000130200081302000813020008130200080C
:10008000130200081302000813020008252C0008C0
:10009000512C0008612C0008130200084964000874
:1000A00013020008130200081302000813020008DC
:1000B0001D6500081302000813020008130200085F
:1000C00013020008130200081302000813020008BC
:1000D00013020008130200081302000813020008AC
:1000E000AD640008130200081302000813020008A0
:1000F000130200081302000813020008130200088C
:10010000130200081302000813020008130200087B
:10011000130200081302000813020008130200086B
:10012000130200081302000813020008130200085B
:10013000130200081302000813020008130200084B
:100140001302000813020008130200085D5900089A
:10015000130200081302000813020008130200082B
:10016000130200081302000813020008130200081B
:10017000130200081302000813020008130200080B
:1001800013020008130200081302000813020008FB
:1001900013020008130200081302000813020008EB
:1001A00013020008130200081302000813020008DB
:1001B00013020008130200081302000813020008CB
:1001C00013020008130200081302000813020008BB
:1001D00013020008130200081302000813020008AB
:1001E000130200081302000813020008130200089B
:1001F000130200081302000813020008130200088B
:100200003D16000800000000000000000000000093
:1002100002E000F000F8FEE772B6374880F3088885
:10022000364880F3098836483649086040F20000B5
:10023000CCF200004EF63471CEF200010860BFF33C
:100240004F8FBFF36F8F40F20000C0F2F0004EF608
:100250008851CEF200010860BFF34F8FBFF36F8F5C
:100260004FF00000E1EE100A4EF63C71CEF20001B4
:100270000860062080F31488BFF36F8F04F0CCFF72
:1002800005F02EFF4FF055301F491B4A91423CBFED
:1002900041F8040BFAE71D49184A91423CBF41F866
:1002A000040BFAE71A491B4A1B4B9A423EBF51F80E
:1002B000040B42F8040BF8E700201849184A914251
:1002C0003CBF41F8040BFAE704F0E4FF05F05CFFE3
:1002D000144C154DAC4203DA54F8041B8847F9E777
:1002E00000F042F8114C124DAC4203DA54F8041BF2
:1002F0008847F9E704F0CCBF000700200023002066
:100300000000000808ED00E00001002000070020C8
:10031000B86A000800230020CC230020D02300204E
:100320006C560020000200080402000804020008C5
:10033000040200082DE9F04F2DED108AC1F80CD011
:10034000D0F80CD0BDEC108ABDE8F08F002383F309
:1003500011882846A047002004F046FAFEE704F082
:10036000C5F900DFFEE70000F8B501F0CDF904F0B3
:10037000CDFE074604F03CFF0546002839D1234B4B
:100380009F4236D001339F4236D0214B27F0FF02E7
:100390009A4234D1F8B200F06FFF2E4642F2107448
:1003A00000F070FF08B10024264601F05FFD20B187
:1003B000032000F083F80024264635B1154B9F42F8
:1003C00003D004F00DFF00242646002004F0A8FE10
:1003D000114B1B695B0416D40EB100F085F801F0D7
:1003E000F5FA00F0BBFF204600F01EF900F07CF8A3
:1003F000F9E72E460024D3E704460126D0E7064657
:100400004FF47A74CCE70024E9E700BF010007B09D
:10041000000008B0263A09B00008024008B501F013
:1004200045F9A0F120035842584108BD07B541F2F3
:100430001203022101A8ADF8043001F055F903B010
:100440005DF804FB38B5302383F31188174803683F
:100450000BB104F095FA164A144800234FF47A7150
:1004600004F084FA002383F31188124C236813B13B
:100470002368013B2360636813B16368013B6360D9
:100480000D4D2B7833B963687BB9022001F008FA6F
:10049000322363602B78032B07D163682BB90220CA
:1004A00001F0FEF94FF47A73636038BDD023002069
:1004B00045040008F0240020E8230020084B1870B1
:1004C00003280CD8DFE800F008050208022001F03C
:1004D000DFB9022001F0D2B9024B00225A60704706
:1004E000E8230020F0240020F8B501F0BFFC30B173
:1004F000454B03221A70454B00225A60F8BD444B0D
:10050000444A1C4619680131F8D004339342F9D1AA
:100510006268414B9A42F1D9404B9B6803F10063FA
:1005200003F580339A42E9D204F02EFE04F040FE37
:10053000002001F003F90220FFF7C0FF384B002133
:100540001A6C19641A6E19661A6E5A6C59645A6ECE
:1005500059665A6E5A6942F080025A615A6922F00D
:1005600080025A615A691A6942F000521A611A6986
:1005700022F000521A611B6972B64FF0E023C3F8F3
:10058000084DD4E90004BFF34F8FBFF36F8F254AA6
:10059000C2F88410BFF34F8F536923F48033536143
:1005A000BFF34F8FD2F88030C3F3C905C3F34E3386
:1005B0005B0143F6E07603EA060C29464CEA8177B4
:1005C0000139C2F87472F9D2203B13F1200FF2D135
:1005D000BFF34F8FBFF36F8FBFF34F8FBFF36F8F9B
:1005E000536923F4003353610023C2F85032BFF340
:1005F0004F8FBFF36F8F302383F31188854680F3CD
:10060000088820477AE700BFE8230020F024002074
:100610000000010820000108FFFF0008002300205F
:100620000038024000ED00E02DE9F04F93B0B74BE9
:1006300000902022FF210AA89D6801F071F9B44AB8
:100640001378A3B9B348012103601170302383F3F9
:10065000118803680BB104F093F9AF4AAD48002349
:100660004FF47A7104F082F9002383F31188009B20
:1006700013B1AA4B009A1A60A94A009C1378032B65
:100680001EBF00231370A54A4FF0000A18BF536025
:10069000D3465646D146012001F0FAF824B19F4BCB
:1006A0001B68002B00F02B82002000F0FFFF03905E
:1006B000039B002B01DA00F099FE039B002BEDDB7E
:1006C000012001F0DBF8039B213B1F2BE3D801A2A3
:1006D00052F823F0550700087D07000811080008AC
:1006E000970600089706000897060008A308000868
:1006F000730A00088D090008EF090008170A0008AE
:100700003D0A0008970600084F0A000897060008EF
:10071000C10A0008F507000897060008050B000845
:1007200061070008F507000897060008EF090008B0
:100730009706000897060008970600089706000825
:100740009706000897060008970600089706000815
:10075000110800080220FFF761FE002840F0F9812F
:10076000009B0221BAF1000F08BF1C4605A841F208
:100770001233ADF8143000F0B7FF8CE74FF47A7005
:1007800000F094FF071EEBDB0220FFF747FE002876
:10079000E6D0013F052F00F2DE81DFE807F0030A13
:1007A0000D10133605230593042105A800F09CFFC6
:1007B00017E056480421F9E75A480421F6E75A4859
:1007C0000421F3E74FF01C08404600F0B9FF08F1A0
:1007D00004080590042105A800F086FFB8F12C0F4D
:1007E000F2D1012000FA07F747EA0B0B5FFA8BFB07
:1007F0004FF0000901F0E0F826B10BF00B030B2BD2
:1008000008BF0024FFF712FE45E748480421CDE762
:10081000002EA5D00BF00B030B2BA1D10220FFF76C
:10082000FDFD074600289BD0012000F087FF022035
:10083000FFF744FE00261FFA86F8404600F08EFFC0
:100840000446B0B10399A1F14002514251414046E2
:1008500000F09CFF01360028EDD1BA46044641F273
:100860001213022105A8ADF814303E4600F03CFFFB
:1008700011E70120FFF722FE2546244B9B68AB427F
:1008800007D9284600F05CFF013040F0678104354D
:10089000F3E7234B00251D70204BBA465D603E46B2
:1008A000A8E7002E3FF45CAF0BF00B030B2B7FF49B
:1008B00057AF0220FFF702FE322000F0F7FEB0F142
:1008C0000008FFF64DAF18F003077FF449AF0F4A59
:1008D000926808EB050393423FF642AFB8F5807F7C
:1008E0003FF73EAF124B0193B84523DD4FF47A70CA
:1008F00000F0DCFE0390039A002AFFF631AF019B63
:10090000039A03F8012B0137EDE700BF0023002015
:10091000EC240020D023002045040008F02400200F
:10092000E823002004230020082300200C230020BB
:10093000EC230020C820FFF771FD074600283FF494
:100940000FAF1F2D11D8C5F1200242450AAB25F08B
:10095000030028BF424683490192184400F0BAFFC1
:10096000019A8048FF2100F0DBFF4FEAA8037D4990
:100970000193C8F38702284600F0DAFF06460028F4
:100980003FF46DAF019B05EB830533E70220FFF7D2
:1009900045FD00283FF4E4AE00F018FF00283FF4C6
:1009A000DFAE0027B846704B9B68BB4218D91F2F9B
:1009B00011D80A9B01330ED027F0030312AA134467
:1009C00053F8203C05934046042205A901F006FA9D
:1009D00004378046E7E7384600F0B2FE0590F2E7BC
:1009E000CDF81480042105A800F07EFE02E7002364
:1009F000642104A8049300F06DFE00287FF4B0AEDB
:100A00000220FFF70BFD00283FF4AAAE049800F087
:100A1000C5FE0590E6E70023642104A8049300F0D6
:100A200059FE00287FF49CAE0220FFF7F7FC002857
:100A30003FF496AE049800F0C1FEEAE70220FFF70B
:100A4000EDFC00283FF48CAE00F0D0FEE1E7022080
:100A5000FFF7E4FC00283FF483AE05A9142000F062
:100A6000CBFE04210746049004A800F03DFE394661
:100A7000B9E7322000F01AFE071EFFF671AEBB0781
:100A80007FF46EAE384A926807EB090393423FF653
:100A900067AE0220FFF7C2FC00283FF461AE27F0EA
:100AA00003074F44B9453FF4A5AE484600F048FE61
:100AB0000421059005A800F017FE09F10409F1E7EB
:100AC0004FF47A70FFF7AAFC00283FF449AE00F01B
:100AD0007DFE002844D00A9B01330BD008220AA9CE
:100AE000002000F025FF00283AD02022FF210AA88C
:100AF00000F016FFFFF79AFC1C4803F07BFE13B0D2
:100B0000BDE8F08F002E3FF42BAE0BF00B030B2B48
:100B10007FF426AE0023642105A8059300F0DAFDDA
:100B2000074600287FF41CAE0220FFF777FC8046C2
:100B300000283FF415AEFFF779FC41F2883003F04E
:100B400059FE059800F06AFF464600F035FF3C4626
:100B5000A1E506464EE64FF0000901E6BA467EE6FC
:100B600037467CE6EC23002000230020A08601000D
:100B7000094A136849F2690099B21B0C00FB013362
:100B80001360064B186844F2506182B2000C01FBFE
:100B90000200186080B27047182300201423002040
:100BA00010B500211022044600F0BAFE034B03CB1F
:100BB000206061601868A06010BD00BF107AF01F4F
:100BC0002DE9F041ADF54E7D0DF134086CAC40F2ED
:100BD000751207460D460EA80021C8F8001000F057
:100BE0009FFE4FF4C4720021204600F099FE02F0EF
:100BF0006BF8254B4FF47A72B0FBF2F0186093E873
:100C00000700022384E807000DF5E9702382FFF74F
:100C1000C7FF40F204431D49238406A805F08EFD5A
:100C2000182384F832310DF2E3266B440DF1300CB9
:100C30001A4603CA624530607160134606F1080621
:100C4000F6D141460122204600F0EAFE002303933C
:100C5000AB7E029305F11903019380B20123CDE924
:100C600004800093E97E06A3D3E90023384602F00E
:100C7000F3FB0DF54E7DBDE8F08100BFAFF30080C2
:100C80009E6AC421818A46EEF82400204C67000841
:100C90002DE9F0412C4C237ADAB080460D465BBB3F
:100CA00027A9284600F0CCFF0746002842D19DF82E
:100CB0009D60C82E3ED801464FF4A662204600F043
:100CC0002FFE4FF48073C4F8F8314FF40073C4F86A
:100CD0000C334FF44073C4F8203432460DF19E01BA
:100CE00004F1090000F0F6FD26449DF89C3077726F
:100CF00023720BB9EB7E23728122002106AC27A858
:100D000000F00EFE0122214627A800F0D5FF0023A7
:100D10000393AB7E029305F1190380B2019328235C
:100D2000CDE904400093E97E05A3D3E900234046C2
:100D300002F092FB5AB0BDE8F08100BFAFF3008033
:100D400026417272DF25D7B718460020F0B5254E30
:100D50004FF48A7505FB0065F1B096F8D83085F838
:100D6000DC300024D822214685F8E8403AA800F07B
:100D7000D7FD06F1090000F0CBFDD5F8E4308DF881
:100D8000F000C2B206AF06F109010DF1F100CDE9A4
:100D90003A3400F09FFD394601223AA800F0B8FF2E
:100DA00080B2CDE9047008230127CDE9023706F1AE
:100DB000D803019330230093317A0B4807A3D3E97A
:100DC000002302F049FBA04206DD01F07DFFC5F8DB
:100DD000E000384671B0F0BD2046FBE778F6339F5F
:100DE00093CACD8D18460020103500202DE9F04122
:100DF0001D4D1E4E1E4F86B0284602F059FB03467D
:100E000058B30024CDE90344ADF81440027B8DF8BB
:100E1000142099684068029403AA03C21B68DFF893
:100E2000548043F00043029301F050FF821941F1D6
:100E30000003009402A9384601F0FAF9A04205DD4A
:100E4000284602F039FB88F80040D5E798F80030D2
:100E5000072B05D8013388F8003006B0BDE8F081D3
:100E6000014802F029FBF8E71035002040420F004E
:100E7000403500204D4B002070B50D4614461E46EF
:100E800002F046FA50B9022E10D1012C0ED112A355
:100E9000D3E90023C5E90023012007E0282C10D066
:100EA00005D8012C09D0052C0FD0002070BD302CA6
:100EB000FBD10BA3D3E90023ECE70BA3D3E9002379
:100EC000E8E70BA3D3E90023E4E70BA3D3E900236E
:100ED000E0E700BFAFF30080401DA12026812A0B70
:100EE00078F6339F93CACD8D9E6AC421818A46EEDF
:100EF00026417272DF25D7B7F017304A39059E5662
:100F000038B505460E4C0021013500F03FFCA4F831
:100F10002C55B4F82C0500F021FC78B1B4F82C0560
:100F200000F02CFC014648B9B4F82C0500F02EFC6A
:100F3000B4F82C350133A4F82C35EAE738BD00BFEE
:100F40001846002010B50A4B0A4A1A6003F5805370
:100F500093F860203AB9DC6D2CB1204601F008F816
:100F6000204605F02BFBBDE81040034801F000B817
:100F700040350020D0670008884500202DE9F04F5B
:100F80008FB000AF05460C4602F0C2F9002849D1E7
:100F9000237E022B1BD1E38A012B18D101F094FE92
:100FA0000646FFF7E5FD03464FF4C870DFF8C4823C
:100FB000B3FBF0F206F5167602FB103316FA83F354
:100FC000C8F80030E37E33B9A34B00221A703C37D7
:100FD000BD46BDE8F08F07F12401204600F0EEFD8C
:100FE0000028F4D107F11400FFF7DAFD97F8264046
:100FF00007F11401224607F1270005F029FB00281C
:10100000E2D10F2C08D8944B1C70D8F80030A3F50F
:101010001673C8F80030DAE797F82410284602F073
:101020006FF9D4E7E38A282B2BD010D8012B23D0DB
:10103000052BCCD1BFF34F8F8849894BCA6802F486
:10104000E0621343CB60BFF34F8F00BFFDE7302B4F
:10105000BDD1844EE17E327A9142B8D1607E314674
:10106000002291F8DC50854200F0A5800132042A6C
:1010700001F58A71F5D1AAE721462846FFF7A0FDC0
:10108000A5E721462846FFF703FEA0E7B2F8EC509B
:101090007B6005F103094FEA99094FEA8902D11DE6
:1010A000C908A8EBC1039D46EB460021584600F055
:1010B00037FC04F1EE012A463144584600F00AFCA0
:1010C0007B6813B9012000F039FB96F8D20000F0DC
:1010D00045FB044630B9307200F078FB204600F042
:1010E0002DFBB1E0D6F8D4203AB996F8D200B6F884
:1010F0002C25824201D8FFF703FFD6F8D4202A44DA
:10110000944208D296F8D200B6F82C2501308242DB
:1011100001D8FFF7F5FE70685FFA89F2594600F0D2
:1011200007FC08B9C54679E0726896F8D2002A44EF
:101130007260D6F8D42005EB0209C6F8D49000F00E
:101140000DFB814509D396F8D220D6F8D4000132A0
:10115000001B86F8D220C6F8D400FF2D0FD800243B
:10116000347200F033FB204600F0E8FA00F07EFE17
:101170003D4B188108B9FFF7B7F9C54627E7BB68AB
:1011800096F8D9000AFB0362FB68D2F8E41082F8F3
:10119000E83001F58061C2F8E030C2F8E410FFF7F2
:1011A000D5FDFFF723FE96F8D920013202F00302A5
:1011B00086F8D920B6E74FF48A7A0AFB02F505F1E2
:1011C000EA013144204600F0CFFDF86000287FF4AA
:1011D000FEAE3544012285F8E82001F075FDD5F812
:1011E000E020D6ED007ADFED216A801A192838BF99
:1011F000192040F6B832904228BF1046B8EE677A00
:1012000007EE900AF8EEE77A67EEA67ADFED186A45
:10121000E7EE267AFCEEE77AC6ED007A96F8D9304A
:10122000BB60BA6873680AFB02F4321992F8E810DE
:1012300059B1D2F8E4108B42E8463FF427AF0021C1
:1012400082F8E810C2F8E010C5467368064A9B0AA7
:1012500001331381BBE600BF0935002000ED00E03B
:101260000400FA0518460020F8240020CDCCCC3D1F
:101270006666663F0C350020014B1870704700BF52
:101280000425002030B54FF000542B4B22689A42C1
:1012900085B007D003F0B6FF044620BB00242046EB
:1012A00005B030BD254B627D25481A70237D037241
:1012B0004FF48073C0F8F8314FF40073C0F80C336A
:1012C00000254FF44073C0F820341E49C0F8E450A4
:1012D000C922093000F0FEFA2046E022294600F03B
:1012E0001FFB0124DBE7184A184D136C43F0007311
:1012F0001364AA6D164B9A42D0D12B6E013B7E2B04
:10130000CCD8144A07CA01AB83E80700184603216A
:1013100000F07AFD6B6D83424FF00003BED12A6D61
:101320008A4201BFAB65054B2A6E1A7003BF0A4B98
:10133000EA6D1A601C46B2E79AAD44C50425002048
:1013400018460020160000200038024000660040C9
:101350005041A0B0586600401023002037B51A4D08
:1013600000F084FD02236B71184B2881196818481E
:10137000012201F045FB00230193164B164900930F
:101380001648174B4FF4805201F092FF154B197815
:1013900011B1124801F0B4FF01F096FC0446FFF7CA
:1013A000E7FB4FF4C873B0FBF3F202FB130304F541
:1013B000167010FA83F00C4B186003F019FF08B197
:1013C0000F232B8103B030BDF82400201023002010
:1013D00040350020790E0008082500201035002037
:1013E0007D0F0008042500200C3500202DE9F04F6A
:1013F0002DED028B0FF23829D9E90089834C93B087
:101400000BAE9FED7E8BFFF7F1FC814FDFF828A23A
:1014100000230A93ADF834300B9373604FF0000B48
:101420005B468DED008B01250DF11D0207A93846A5
:101430008DF81C508DF81DB001F090FA9DF81C300D
:10144000002B40F0A580204601F062FF06460028F0
:1014500045D1704F01F038FC3B6898423FD301F012
:1014600033FC8246FFF784FB4FF4C873B0FBF3F202
:1014700002FB13030AF5167010FA83F03860664F0A
:1014800097F800B0CBF1100ABBF1000F14BF334640
:101490002B465FFA8AFA0EA88DF82830FFF780FBFA
:1014A000BAF1060F28BF4FF0060A0EAB03EB0B0193
:1014B00052460DF1290000F00DFA0AAB03931823F0
:1014C00002930AF10102554BD2B2CDE900530492C6
:1014D00020464CA3D3E9002301F060FF3E7001F0E9
:1014E000F3FB4F4A4F4D1368C31AB3F57A7F2ED3DF
:1014F000106001F0EBFB02460B46204601F0E6FFD0
:10150000204601F005FF10B32B7A474E002B14BF85
:1015100003230223737101F0D7FB0EAF4FF47A73EC
:101520000122B0FBF3F039463060304600F01EFB7C
:10153000182302933D4B019380B240F25513CDE93D
:101540000370009342464B46204601F027FF2B7A5A
:1015500093B101F0B9FB002607464FF48A7A95F85B
:10156000D900304400F003000AFB005393F8E82050
:1015700092B30136042EF2D1C82003F03BF92B7A46
:10158000002B7FF43DAF13B0BDEC028BBDE8F08FB4
:10159000DAF8143083F04003CAF8143059461022A8
:1015A0000EA800F0BDF90DF11E0308AA0AA93846DD
:1015B00000F03EFF96E803000FAB83E803009DF8C0
:1015C00034308DF844300A9B0E930EA9DDE90823D0
:1015D000204602F04FF921E7D3F8E02042B12B6812
:1015E000FA2B38BFFA23BA1A0533B2EB430FC0D334
:1015F000FFF7ACFB0028BCD1BEE700BF0000000035
:1016000000000000401DA12026812A0B103500207B
:10161000403500200C350020093500200835002019
:10162000484B002018460020F82400204C4B002096
:10163000F1C6A7C1D068080F0000024008B50548F0
:1016400000F092FFBDE80840034A0449002004F07E
:10165000AFBF00BF40350020884B0020450F000879
:1016600070B50F4B1B780133DBB2012B0C4611D840
:101670000C4D29684FF47A730E6AA2FB03320146BF
:1016800022462846B047844204D1074B00221A70F4
:10169000012070BD4FF4FA7003F0ACF80020F8E7B9
:1016A0001C230020004E00207C4B002007B50023A7
:1016B000024601210DF107008DF80730FFF7D0FF3A
:1016C00020B19DF8070003B05DF804FB4FF0FF3038
:1016D000F9E700000A4608B50421FFF7C1FF80F0D2
:1016E0000100C0B2404208BD30B4054C2368DD693A
:1016F000044B0A46AC460146204630BC604700BF5A
:10170000004E0020A086010070B503F093FB094E47
:10171000094D3080002428683388834208D903F0BB
:1017200083FB2B6804440133B4F5803F2B60F2D374
:1017300070BD00BF7E4B0020504B002003F02ABC40
:1017400000F1006000F580300068704700F1006033
:10175000920000F5803003F0B3BB0000054B1A681F
:10176000054B1B889B1A834202D9104403F05CBBD3
:1017700000207047504B00207E4B0020024B1B681E
:10178000184403F059BB00BF504B0020024B1B68AC
:10179000184403F069BB00BF504B002010F0030356
:1017A0000AD1B0F5047F05D200F10050A0F57920F0
:1017B000D0F80038184670470023FBE700F10050CE
:1017C000A0F57920D0F8100A70470000064991F87A
:1017D000243033B10023086A81F824300822FFF74F
:1017E000B5BF0120704700BF544B0020014B186863
:1017F000704700BF002004E0F0B51E4B1D680138A3
:101800002E0C0A181C48C5F30B0403233546078821
:10181000A7420BD144680B46013C934218461BD2A9
:1018200014F9010F48B103F8010BF6E7013B00F191
:101830000800ECD191420ED20B4618462C24B6F586
:10184000805F00F8014B0AD1824202D94122981CE4
:101850005A70401AF0BD0846B6F5805FF9D041F2E3
:1018600001039D42F5D18242F3D95A2300F8013B8E
:10187000EFE700BF002004E020230020022802BF81
:10188000024B4FF480029A61704700BF0000024093
:10189000022802BF014B40229A61704700000240BB
:1018A000022801BF024A536983F040035361704725
:1018B0000000024070B504464FF47A764CB1412CDA
:1018C000254628BF412506FB05F002F093FF641B67
:1018D000F4E770BD10B50023934203D0CC5CC45430
:1018E0000133F9E710BD000010B5013810F9013FD0
:1018F0003BB191F900409C4203D11AB10131013A48
:10190000F4E71AB191F90020981A10BD1046FCE7CF
:1019100003460246D01A12F9011B0029FAD170477A
:1019200002440346934202D003F8011BFAE77047D2
:101930002DE9F8431F4D144695F8242007468846A4
:1019400052BBDFF870909CB395F824302BB920225D
:10195000FF2148462F62FFF7E3FF95F82400C0F10E
:101960000802A24228BF2246D6B24146920005EBA9
:101970008000FFF7AFFF95F82430A41B1E44F6B299
:10198000082E17449044E4B285F82460DBD1FFF7B9
:101990001DFF0028D7D108E02B6A03EB82038342A6
:1019A000CFD0FFF713FF0028CBD10020BDE8F8838C
:1019B0000120FBE7544B0020024B1A78024B1A70AF
:1019C000704700BF7C4B00201C23002010B5104C3A
:1019D000104802F05DFA21460E4802F085FA2468AC
:1019E000E26ED2F8043843F00203C2F804384FF430
:1019F0007A70FFF75FFF0849204602F07DFBE26E38
:101A0000D2F8043823F00203C2F8043810BD00BF36
:101A1000BC680008004E0020C46800087047000041
:101A20002DE9F0470D46044600219046284640F235
:101A30007912FFF775FF234620220021284601F086
:101A4000BBFE231D02222021284601F0B5FE631DA6
:101A500003222221284601F0AFFEA31D03222521E7
:101A6000284601F0A9FE04F1080310222821284687
:101A700001F0A2FE04F1100308223821284601F0EB
:101A80009BFE04F1110308224021284601F094FE38
:101A900004F1120308224821284601F08DFE04F1CA
:101AA000140320225021284601F086FE04F1180379
:101AB00040227021284601F07FFE04F12003082215
:101AC000B021284601F078FE04F121030822B82154
:101AD000284601F071FE04F12207C0263B4631463C
:101AE00008222846083601F067FEB6F5A07F07F108
:101AF0000107F3D104F1320308223146284601F0F0
:101B00005BFE002704F1330A94F832304FEAC7092C
:101B10009F4209F5A47615D3B8F1000F08D13146DC
:101B200004F599730722284601F046FE09F24F1684
:101B3000274694F832213B1B93420CD3F01DC0087A
:101B4000BDE8F0870AEB070308223146284601F07A
:101B500033FE0137D8E707F233133146082228460F
:101B600001F02AFE08360137E3E7000013B504460A
:101B70000846002101602346C0F80310202201908E
:101B800001F01AFE0198231D0222202101F014FE0B
:101B90000198631D0322222101F00EFE0198A31D6E
:101BA0000322252101F008FE019804F10803102208
:101BB000282101F001FE072002B010BDF7B5002377
:101BC000047F00910E4607221946054601F0B8FC35
:101BD000731C0093012200230721284601F0B0FC6A
:101BE000C4B9B31C0093052223460821284601F0FE
:101BF000A7FC0D243746B278BB1B934211D32B7F31
:101C0000A88A0734E408BBB9844294BF00200120AD
:101C100003B0F0BDAB8ADB00083BDB08B3700824DF
:101C2000E8E7FB1C0093214600230822284601F028
:101C300087FC08340137DEE7201A18BF0120E7E7E8
:101C4000F7B50023047F00910E4608221946054689
:101C500001F076FC731CC4B9082200931146234698
:101C6000284601F06DFC1024012372785F1C013BB3
:101C7000934211D32B7FA88A0734E408BBB984426E
:101C800094BF0020012003B0F0BDAB8ADB00083B0D
:101C9000DB0873700824E7E7F3190093214600235B
:101CA0000822284601F04CFC08343B46DDE7201AA8
:101CB00018BF0120E7E70000F8B50E4605461446B8
:101CC000002181223046FFF72BFE2B4608220021FF
:101CD000304601F071FD7CB96B1C072208213046AB
:101CE00001F06AFD0F2401236A785F1C013B9342D7
:101CF00004D3E01DC008F8BD0824F4E7EB19214621
:101D00000822304601F058FD08343B46ECE700005D
:101D1000F8B50E46054614460021CE223046FFF7A0
:101D2000FFFD2B4628220021304601F045FD7CB9FD
:101D300005F1080308222821304601F03DFD30243A
:101D40002F462A7A7B1B934204D3E01DC008F8BDBE
:101D50002824F5E707F1090321460822304601F05F
:101D60002BFD08340137ECE7F7B5047F00910E46F0
:101D7000012310220021054601F0E2FBC4B9B31C87
:101D80000093092223461021284601F0D9FB19248B
:101D900037467288BB1B9A4211D82B7FA88A07341A
:101DA000E408BBB9844294BF0020012003B0F0BD19
:101DB000AB8ADB00103BDB0873801024E8E73B1D97
:101DC0000093214600230822284601F0B9FB08347D
:101DD0000137DEE7201A18BF0120E7E730B5094DCB
:101DE0000A4491420DD011F8013B5840082340F3BA
:101DF0000004013B2C4013F0FF0384EA5000F6D1AD
:101E0000EFE730BD2083B8EDF7B54FF0FF33DFF8D3
:101E100054C0DFF854E000EB81011A4688421CD020
:101E200050F8044B019401AF042417F8015B82EAD7
:101E300005620825DB18164605F1FF355241002ED4
:101E4000BCBF83EA0C0382EA0E0215F0FF05F1D154
:101E5000013C14F0FF04E8D1E0E7D843D14303B0DC
:101E6000F0BD00BF9336EAA9EBE1F042F7B53A4A7C
:101E7000106851686B4603C36A46384938480823DE
:101E800004F0F6FB0446002835D10A25354A1068CF
:101E900051686B4603C36A4633493148082304F04E
:101EA000E7FB044600284DD00369B3F5E02F49D87D
:101EB000B0F8662040F204418A4201D0552A41D14F
:101EC0002A4A224402F15C018B423BD35C3B244909
:101ED00000209E1AFFF782FF3246074604F1640194
:101EE0000020FFF77BFFA3689F422BD1E368984255
:101EF00008BF002526E00369B3F5E02F29D8428BFF
:101F000040F204418A4201D0552A20D1174A224486
:101F100002F110018B4218D3103B114900209D1A89
:101F2000FFF75CFF2A46064604F118010020FFF780
:101F300055FFA3689E4202D1E368984201D00D2567
:101F4000A4E70025284603B0F0BD10259EE70C2528
:101F50009CE70B259AE700BF94670008DCFF0600AA
:101F6000000001089D67000890FF06000800FFF7C9
:101F700010B5037C044613B9006804F061FB2046E9
:101F800010BD00000023BFF35B8FC360BFF35B8F06
:101F9000BFF35B8F8360BFF35B8F7047BFF35B8FD3
:101FA0000068BFF35B8F704770B505460C30FFF7D4
:101FB000F5FF05F1080604463046FFF7EFFFA042A3
:101FC00006D930466D68FFF7E9FF2544281A70BD31
:101FD0003046FFF7E3FF201AF9E7000070B5054629
:101FE000406898B105F10800FFF7D8FF05F10C062D
:101FF00004463046FFF7D2FF8442304694BF6D68F6
:102000000025FFF7CBFF013C2C44201A70BD0000D7
:1020100038B50C460546FFF7C7FFA04210D305F1BF
:102020000800FFF7BBFF04446868B4FBF0F100FB55
:102030001144BFF35B8F0120AC60BFF35B8F38BDF1
:102040000020FCE72DE9F041144607460D46FFF756
:10205000C5FF844228BF0446D4B1B84658F80C6B7B
:102060004046FFF79BFF3044286040467E68FFF7FC
:1020700095FF331A9C4203D86C600120BDE8F081C3
:102080006B60A41B3B68AB602044E8600220F5E76E
:102090002046F3E738B50C460546FFF79FFFA04200
:1020A00010D305F10C00FFF779FF04446868B4FB16
:1020B000F0F100FB1144BFF35B8F0120EC60BFF334
:1020C0005B8F38BD0020FCE72DE9FF41884669465B
:1020D0000746FFF7B7FF6C4606B204EBC6060025BD
:1020E000B44209D06268206808EB0501FFF7F2FBF3
:1020F000636808341D44F3E729463846FFF7CAFFF2
:10210000284604B0BDE8F081F8B505460C300F460E
:10211000FFF744FF05F1080604463046FFF73EFF8F
:10212000A042304688BF6C68FFF738FF201A38603D
:1021300020B130462C68FFF731FF2044F8BD000085
:1021400073B5144606460D46FFF72EFF844228BF9E
:1021500004460190DCB101A93046FFF7D5FF019B91
:1021600033B93268C5E90233C5E9002401200CE027
:102170009C4238BF01942860019868608442F5D978
:102180003368AB60241AEC60022002B070BD2046B8
:10219000FBE700002DE9FF410F466946FFF7D0FF3E
:1021A0006C4600B204EBC0050026AC4209D0D4F85E
:1021B000048054F8081BB8194246FFF78BFB4644CD
:1021C000F3E7304604B0BDE8F081000038B50546BD
:1021D000FFF7E0FF044601462846FFF719FF2046B7
:1021E00038BD000010B4026854681A4623465DF8F2
:1021F000044B1847002070470020704770470000CC
:10220000002070470E20704700F5805090F8C800FD
:10221000C0F340007047000000F5805090F9D000F6
:102220007047000000F58050C0F8CC1001207047C6
:10223000F7B50C68BDF8207014F0005470D10D7B18
:10224000082D6DD8302585F311884569AE68760173
:102250000CD4AC68240108D4AC6814F080545DD16F
:1022600084F31188204603B0F0BD01240E6804F108
:10227000180C002EB8BFF6004FEA0C1CB4BF46F095
:102280000406760545F80C600E680FFA84FC16F01B
:10229000804F18BF05EB0C1E05EB0C1C1EBFDEF8B3
:1022A000806146F00206CEF880610E7BCCF8846136
:1022B00005EB04158E68C5F88C614E68C5F8886119
:1022C000DCF8805145F00105CCF8805100EB441654
:1022D00041F268052E4405EB44150544C6E9002388
:1022E00008350E4601F10C0C56F804EB45F804EBEA
:1022F0006645F9D1843436882E8000EB441407F00B
:102300000305267926F00B0635432571002484F356
:102310001188009700F0FAFC0120A4E70224A5E749
:102320004FF0FF309FE7000013B500F58054019196
:10233000E06DFFF753FE1F280AD90199E06D2022B6
:10234000FFF7C2FEA0F120035842584102B010BD71
:102350000020FBE708B5302383F3118800F5805097
:10236000C06DFFF70FFE002383F3118808BD000046
:1023700000220260828142608260704710B50022B4
:102380000023C0E900230023044603810C30FFF73B
:10239000EFFF204610BD0000F0B5054600F5805067
:1023A0000C4690F8C83013F0040FC3F3800108BF47
:1023B000114661F3820304F1840680F8C83005EB0E
:1023C000461389B01B79D8072ED57AB319072DD4B7
:1023D0006846FFF7D3FF05EB441303F5835303F17E
:1023E000180703AA103318685968144603C4083341
:1023F000BB422246F7D1186820609B88A380DDE9A4
:102400000E23CDE900230123ADF808302B6869467F
:10241000DB6B2846984705EB46152B791A075CBFFE
:1024200043F008032B7101E0002AF4D109B0F0BD9C
:102430002DE9F0479A4688B00746884691463023F2
:1024400083F3118807F580546846FFF797FFE06D26
:10245000FFF7AAFD1F282AD9E06D20226946FFF761
:10246000B5FE202823D103AD444605AB2E4603CE4E
:102470009E4220606160354604F10804F6D1306860
:102480002060B388A380DDE90023C9E90023BDF8FB
:102490000830AAF80030002383F3118853464A46D7
:1024A0004146384608B0BDE8F04700F01DBC0020AA
:1024B00080F3118808B0BDE8F08700002DE9F84FDF
:1024C0000023C0E90133254B044640F8183B0F4672
:1024D000FFF74EFF04F12800FFF750FF04F1480812
:1024E00004F582554646083530462036FFF746FF4C
:1024F000AE42F9D104F580554FF480534FF00009F6
:10250000C5E91339C5F848800123EE6504F58758FD
:1025100004F58456C5F8549085F8583085F8603035
:10252000083608F108084FF0000A4FF0000B46E9A2
:1025300008ABA6F11800FFF71BFF203646F8289CD1
:102540004645F4D185F8D07017B1054800F0B6FBC8
:10255000044B63612046BDE8F88F00BFD0670008D8
:10256000A86700080064004010B5044B19780446C1
:102570004A1C1A70FFF7A2FF204610BD844B0020B2
:102580002DE9F04300294FD0284B2948B0FBF1F04A
:1025900099428CBF0A2311235D1EB0FBF3F703FBA6
:1025A0001703ECB22BB1022D2B46F5D80020BDE865
:1025B000F0837E1EB6F5806FF8D2C4EBC40C0CF12C
:1025C00003034FEAE308C3F3C703A4EB030E08F1C8
:1025D00001094FF47A755FFA8EF008FB055559FA38
:1025E0008EFEB5FBFEF5B5F5617FC1BF0CF1FF3383
:1025F000C3F3C703E01AC0B25C1C50FA84F40C4D5C
:102600007C43B5FBF4F4A142D0D1013BDBB20F2BEC
:10261000CCD80138C0B20728C8D800211071168064
:102620009170D3700120C2E70846C0E73F420F0017
:1026300080F9370370B505460E464FF47A746B691E
:102640005B6803F00103B34207D04FF47A7002F0E5
:10265000D1F8013CF3D1204670BD0120FCE7000019
:1026600030B54269936913F0700F16D000230B4CFC
:10267000936103F1840200EB421211794D0709D5F1
:10268000890707D5416954F823508D60117941F0CD
:10269000040111710133032BEBD130BDBC6700087D
:1026A00073B51D46436916469A68D207044609D594
:1026B0009A6801219960C2F34002CDE900650021CA
:1026C000FFF76AFE63699A68D1050BD59A684FF4E3
:1026D00080719960C2F34022CDE900650121204656
:1026E000FFF75AFE63699A68D2030BD59A684FF4D4
:1026F00080319960C2F34042CDE900650221204655
:10270000FFF74AFE04F58053D3F8CC0010B10368FC
:102710001B699847204602B0BDE87040FFF7A0BF94
:10272000F8B504464669002972D106F10C073868ED
:10273000800770D006EB01153868D5F8B00110F0AD
:10274000040FD5F8B0011ABFC00840F00040400D9A
:10275000A061D5F8B0C11CF0020F1CBF40F0804052
:10276000A061D5F8B40106EB011100F00F0084F868
:102770002400D1F8B8012077D1F8B801000A6077B9
:10278000D1F8B801000CA077D1F8B801000EE077BD
:10279000D1F8BC0184F82000D1F8BC01000A84F80B
:1027A0002100D1F8BC01000C84F82200D1F8BC1142
:1027B000090E84F823103821396004F1340004F143
:1027C000180104F1240551F8046B40F8046BA94288
:1027D000F9D109880180C4E90A2321460023238610
:1027E00051F8283B2046DB6B984704F5805393F85B
:1027F000C820D3F8CC0042F0040283F8C82010B1FE
:1028000003681B6998472046BDE8F840FFF728BFDA
:1028100006F110078BE7F8BD10B5044600F056FA34
:1028200002460B4652EA030102D0013A63F100036B
:102830000449086820B12146BDE81040FFF770BF89
:1028400010BD00BF804B0020F0B5302181F311880E
:10285000DFF848C000F583510831002404F18405F5
:1028600000EB45152E7977070ED4F6060CD5D1E985
:10287000007697429E4107D246695CF82470B760A3
:102880002E7946F004062E710134032C01F120014B
:10289000E4D1002383F31188F0BD00BFBC670008BA
:1028A00008B5302383F31188FFF7DAFE002383F3A2
:1028B000118808BDF8B543690546986800F0E050F6
:1028C000B0F1E05F0F4621D0F8B1302383F31188D7
:1028D00005F583541034002606F1840305EB4313F9
:1028E0001B791A0706D50136032E04F12004F3D113
:1028F000012007E05B07F6D42146384600F040FA95
:102900000028F0D1002383F31188F8BD0120FCE7F3
:1029100008B5302383F3118800F58050C06DFFF7B0
:1029200043FB002383F3118843090CBF01200020DF
:1029300008BD0000F8B51D46002313700F4606467B
:102940001446FFF7E5FF80F00100387025B12946F5
:102950003046FFF7AFFF2070F8BD00002DE9B84109
:102960000C4615461F46804600F0B0F90B4621780C
:10297000024609B9287850B14046FFF765FFFFF7D6
:102980008FFF3B462A462146FFF7D4FF0120BDE8D2
:10299000B881000070B5302686F31188174B1A6C89
:1029A00042F000721A641A6A42F000721A621A6ADD
:1029B00022F000721A62002383F3118800F580541C
:1029C00094F8C83013F0010516D1A9B186F3118827
:1029D0000321132001F0CCF90321142001F0C8F9E0
:1029E0000321152001F0C4F994F8C83043F0010325
:1029F00084F8C83085F3118870BD00BF00380240EC
:102A00002DE9F04700F5805588B095F8D030012BBE
:102A100004468846164600F28180814F57F82320ED
:102A20000AB947F82300D7F800A0C4F80C80267430
:102A3000BAF1000F64D095F8D030012B70D001218D
:102A40002046FFF7A7FF302383F3118862691368DC
:102A500023F0020313606269136843F001031360FB
:102A6000636900275F6187F3118801212046FFF722
:102A7000E1FD002800F09580E86DFFF783FA04F58A
:102A80008359BA4609F10809202200216846FEF759
:102A900047FF02A8FFF76CFCCDF818A06A4609EBC7
:102AA00007030DF1180E9446BCE80300F4451860C6
:102AB0005960624603F10803F5D1DCF800001860A4
:102AC00020379CF804201A71602FDDD195F8C830AA
:102AD0006FF38203002785F8C8306A4641462046D6
:102AE000ADF80070ADF802708DF80470FFF748FD86
:102AF000636948BB4FF400421A6008B0BDE8F08734
:102B000041F2D80003F05CFD814610B15146FFF759
:102B1000D5FCC7F80090B9F1000F8CD10020ECE78C
:102B2000386803681B6B98470146002887D13868CE
:102B3000FFF730FF3868036832465B6841469847C4
:102B400000287FF47CAFE9E761221A609DF802302B
:102B50009DF803201B06120402F4702203F0407358
:102B60001343BDF80020C2F3090213439DF804206B
:102B70001205022E02F4E0020CBF4FF000410021CA
:102B8000134362690B43D361636913225A6162691B
:102B9000136823F00103136039462046FFF74AFD0E
:102BA00008B96369A6E795F8D03093BB6169D1F89D
:102BB000002242F00102C1F800226169D1F800222E
:102BC00022F47C5222F00E02C1F800226169D1F891
:102BD000002242F46062C1F800226269C2F8143235
:102BE0006269C2F80432626941F6FF71C2F80C12E0
:102BF0006269C2F840326269C2F8443263690122F4
:102C0000C3F81C226269D2F8003223F00103C2F833
:102C1000003295F8C83043F0020385F8C8306CE7FD
:102C2000804B002008B500F051F850EA010302463D
:102C300002D0421E61F10001044B186810B10B462E
:102C4000FFF72EFDBDE8084001F068B8804B00207A
:102C500008B50020FFF7E0FDBDE8084001F05EB8D0
:102C600008B50120FFF7D8FDBDE8084001F056B8CF
:102C700000B59BB0EFF3098168226846FEF72AFE93
:102C8000EFF30583014B9B6BFEE700BF00ED00E017
:102C900008B5FFF7EDFF000000B59BB0EFF3098129
:102CA00068226846FEF716FEEFF30583014B5B6B67
:102CB000FEE700BF00ED00E0FEE700000FB408B53E
:102CC000029801F03DFDFEE702F0BEB902F0A0B9A6
:102CD00013B56C4684E80600031D94E8030083E8FE
:102CE0000500012002B010BD73B58568019155B192
:102CF0001B885B0707D4D0E900369B6B9847019A85
:102D0000C1B23046A847012002B070BDF0B5866858
:102D100089B005460C465EB1BDF838305B070AD471
:102D2000D0E900379B6B98472246C1B23846B0477E
:102D3000012009B0F0BD00220023CDE900230023CB
:102D4000ADF808300A4603AB01F108061068516877
:102D50001C4603C40832B2422346F7D110682060F3
:102D60009288A280FFF7B2FF0423ADF808302B68E9
:102D7000CDE90001DB6B694628469847D8E700009B
:102D800030B503680968DD0FB5EBD17F23F06044EF
:102D900021F060424FEAD1700BD0002BB8BFA40CD9
:102DA0000029B8BF920C944202D034BF0120002009
:102DB00030BD944205D1C1F38070C3F38073834268
:102DC000F6D194422CBF00200120F1E72DE9F0411B
:102DD000456A15B94162BDE8F0814B6823F0604750
:102DE000C3F38A464FEAD37EC3F3807816EA2306FC
:102DF00038BF3E46AC462B465A68BEEBD27F22F027
:102E000060440AD0002A18DAA40CB44217D19D42BB
:102E10000FD10D60DEE71346EEE7A74207D102F0BF
:102E20008044C2F3807242450BD054B1EFE708D220
:102E3000EDE7CCF800100B60CDE7B44201D0B4420E
:102E4000E5D81A689C46002AE5D11960C3E700005E
:102E50002DE9F047089D01F007044FEAD508224408
:102E600005F0070500EBD1004FF47F49944201D1F2
:102E7000BDE8F08704F0070705F0070A57453E460E
:102E800038BF5646C6F10806111B8E4228BF0E46B3
:102E9000E10808EBD50E415C13F80EC0B94029FAE1
:102EA00006F721FA0AF1FFB28CEA010147FA0AF7A4
:102EB00039408CEA010C03F80EC034443544D5E7A0
:102EC00080EA0120082341F2210201B240000029DA
:102ED00080B203F1FF33B8BF504013F0FF03F4D1C9
:102EE0007047000038B50C468D18A54200D138BD9A
:102EF00014F8011BFFF7E4FFF7E7000042684AB14E
:102F0000136843604389818901339BB299424381AD
:102F100038BF83811046704770B588B020220446C0
:102F20000D4668460021FEF7FBFC20460495FFF79E
:102F3000E5FF024658B16B46054608AE1C4603CC79
:102F4000B44228606960234605F10805F6D11046B1
:102F500008B070BD082817D909280CD00A280CD051
:102F60000B280CD00C280CD00D280CD00E2814BF28
:102F70004020302070470C207047102070471420EC
:102F8000704718207047202070470000082817D984
:102F90000C280CD910280CD914280CD918280CD9B5
:102FA00020280CD930288CBF0F200E207047092014
:102FB00070470A2070470B2070470C2070470D2087
:102FC000704700002DE9F843078C072F04461ED9EF
:102FD000D0E9029800254FF6FF73C5F12006A5F150
:102FE000200029FA05F108FA06F628FA00F0314324
:102FF0000143C9B21846FFF763FF0835402D034669
:10300000EBD1E1693A46BDE8F843FFF76BBF4FF6F5
:10301000FF70BDE8F883000010B54B6823B9CA8A79
:1030200063F30902CA8210BD04691A681C60036157
:10303000C38A013BC3824A60EFE700002DE9F84FE5
:103040001D46CB8A0F46C3F30901052981469246E6
:103050000B4630D00020AAB207F11A049EB2042E0B
:103060001FFA80F80FD8904503F1010306D3FB8ABD
:103070000A4462F30903FB8201201AE01AF8006097
:10308000E6540130EAE79045F1D2A1F1050B1C238B
:103090007C68BBFBF3F203FB12BB1FFA8BF6002C20
:1030A00045D14846FFF72AFF044638B978606FF0EB
:1030B0000200BDE8F88F4FF00008E6E70026066042
:1030C0007860ADB24FF0000B454510D90AEB08030C
:1030D000221D13F8011B9155B1B208F101081B29FB
:1030E0001FFA88F82BD0454506F10106F1D8FB8A76
:1030F000C3F30902154465F30903BCE7013292B238
:103100001C462368002BF9D16B1F0B441C21B3FB19
:10311000F1F301339BB29A42D3D2BBF1000FD0D16D
:103120004846FFF7EBFE20B9C4F800B0BFE7012224
:10313000E7E7C0F800B05E4620600446C1E74545B9
:10314000D5D94846FFF7DAFE08B92060AFE7C0F8E6
:1031500000B0002620600446B6E700002DE9F04FDD
:103160002DED028B1C4683B05B69019207468846B1
:10317000002B00F09A80238C2BB1E269002A00F02A
:103180009480072B35D807F10C00FFF7B7FE0546F2
:1031900038B96FF00205284603B0BDEC028BBDE8DC
:1031A000F08F14220021FEF7BBFB228CE16905F1B0
:1031B0000800FEF78FFB208C013080B2FFF7E6FE9F
:1031C000FFF7C8FE013880B220840130287463699B
:1031D000228C1B782A4403F01F0363F03F0348F05E
:1031E00000411372384669602946FFF7EFFD01255B
:1031F000D1E700F10C034FF0000908EE103A4FF050
:10320000800A4E464D4618EE100AFFF777FE8346B9
:103210000028BED014220021FEF782FB002E3AD1F6
:10322000019BABF8083002220BF1080E1FFA82FC5A
:103230000CF10100BCF1060F218C80B201D88E4246
:103240002BD3FFF7A3FEFFF785FE626912780138E2
:1032500002F01F028E4208BF4FF0400A42EA4912B4
:103260001BFA80F14AEA020A013048F0004281F874
:1032700008A08BF81000CBF8042059463846FFF719
:10328000A5FD238C0135B3422DB289F001094FF021
:10329000000AB8D17FE70022C6E7E169895D0EF830
:1032A00002100136B6B20132C0E76FF0010572E7D5
:1032B000F8B515460E463022002104461F46FEF79B
:1032C0002FFB069B6360B5F5001F079BA76034BF0B
:1032D0006A094FF6FF72A36297B2E66104F110002B
:1032E00000239A4206D800230360A782E382238347
:1032F000E360F8BD0660013330462036F1E7000098
:1033000003781BB94BB2002BC8BF01707047000097
:1033100000787047F8B50C46C969074611B9238C87
:10332000002B37D1257E1F2D34D8387828BB228C2E
:10333000072A2CD8268A36F003032BD14FF6FF70CC
:10334000FFF7D0FD20F001003102400441EA0561A1
:10335000400C41EA40254FF6FF7223462946384685
:10336000FFF7FCFE002807DD626913780133DBB24A
:103370001F2B88BF00231370F8BD218A2D0645EA54
:10338000012505432046FFF71DFE0246E5E76FF0E5
:103390000300F1E76FF00100EEE7000070B58AB0BE
:1033A000044616460021282268461D46FEF7B8FA54
:1033B000BDF83830ADF810300F9B05939DF84030C4
:1033C0008DF81830119B07936946BDF84830ADF869
:1033D00020302046CDE90265FFF79CFF0AB070BDA2
:1033E0002DE9F041D36905460C4616460BB9138CFE
:1033F0005BBB377E1F2F28D895F80080B8F1000FEF
:1034000026D03046FFF7DEFD3378210241EAC33192
:1034100041EA0801338A41EA076141EA0341024671
:10342000334641F080012846FFF798FE00280ADD68
:103430003378012B07D1726913780133DBB21F2B6C
:1034400088BF00231370BDE8F0816FF00100FAE738
:103450006FF00300F7E70000F0B58BB004460D46AF
:1034600017460021282268461E46FEF759FA9DF8A5
:103470004C305A1E534253418DF800309DF8403075
:10348000ADF81030119B05939DF848308DF8183039
:10349000149B07936A46BDF85430ADF82030294696
:1034A0002046CDE90276FFF79BFF0BB0F0BD000090
:1034B000406A00B104307047436A1A684262026988
:1034C0001A600361C38A013BC38270472DE9F04152
:1034D000D0F82080194E14461D464146002709B9F0
:1034E000BDE8F081D1E90223A21A65EB03039642FD
:1034F00077EB03031ED2036A8B420DD1FFF78CFDDD
:10350000036A1B68036203690B60C38A0161016A75
:10351000013BC3828846E2E7FFF77EFD0B68C8F8EF
:10352000003003690B60C38A0161013BC382D8F894
:103530000010D4E788460968D1E700BF80841E00E8
:103540002DE9F04F8BB00D46DDF8509014469B46A8
:103550008046002800F01981B9F1000F00F01581B4
:10356000531E3F2B00F21181012A03D1BBF1000F42
:1035700040F00B810023CDE90833B8F81430B5EBE7
:10358000C30F4FEAC30703D300200BB0BDE8F08F91
:103590002B199F42D8F80C303ABF7F1BFFB2274649
:1035A0001BB9D8F81030002B7AD0272D4ED8C5F192
:1035B0002806B7424FF000032CBFF6B23E460093F8
:1035C0002946D8F8080008AB3246FFF741FCA7EBC4
:1035D000060A35445FFA8AFAB8F8143003F100534A
:1035E000053BDB000493D8F80C3003932821039BA0
:1035F00013B1BAF1000F2CD1D8F8100040B1BAF1D4
:10360000000F05D0009608AB5246691AFFF720FC60
:1036100038B2002FB8D066070AD00AAB03EBD4014A
:10362000624211F8083C02F00702134101F8083C1D
:10363000082C3CD9102C40F2B580202C40F2B780E9
:10364000BBF1000F00F09C80082334E0BA4600264E
:10365000C2E7049BE02B28BFE02306930B44AB4258
:10366000059314D95A1B03980096924534BF5246CD
:10367000D2B2691A08AB04300792FFF7E9FB079A48
:103680001644AAEB020A1544F6B25FFA8AFA049BC2
:10369000069A05999B1A0493039B1B680393A6E75C
:1036A0000093D8F8080008AB3A462946AEE7BBF1CC
:1036B000000F13D00123B4EBC30F6CD0082C12D829
:1036C0009DF82030621E23FA02F2D50706D54FF08E
:1036D000FF3202FA04F423438DF820309DF82030A5
:1036E00089F8003051E7102C12D8BDF82030621E46
:1036F00023FA02F2D10706D54FF0FF3202FA04F4A2
:103700002343ADF82030BDF82030A9F800303CE765
:10371000202C0FD80899631E21FA03F3DA0705D588
:103720004FF0FF3202FA04F40C430894089BC9F8E6
:1037300000302AE7402C2BD0DDE90865611EC4F17A
:103740002102A4F1210326FA01F105FA02F225FA79
:1037500003F311431943CB0712D50122A4F120032F
:10376000C4F1200102FA03F322FA01F1A24052420D
:1037700043EA010363EB430332432B43CDE90823C0
:10378000DDE90823C9E90023FFE66FF00100FCE64C
:103790006FF00800F9E6082CA0D9102CB3D9202C22
:1037A000EED8C3E7BBF1000FADD0022383E7BBF136
:1037B000000FBBD004237EE730B5012A144638BF82
:1037C0000124402C85B028BF40240025012ACDE9E2
:1037D000025518D81B788DF8083063070AD004AB5F
:1037E00003EBD405624215F8083C02F0070293404F
:1037F00005F8083C009103462246002102A8FFF785
:1038000027FB05B030BD082AE4D9102A03D81B884D
:10381000ADF80830E1E7202A8DBFD3E900231B680B
:103820000293CDE90223D8E710B5CB681BB98B60B2
:103830000B618B8210BD04691A681C600361C38A26
:10384000013BC382CA60F0E703064CBFC0F3C0303F
:103850000220704708B50246FFF7F6FF022806D19E
:103860005306C2F30F2001D100F0030008BDC2F3DC
:103870000740FBE72DE9F04F93B0CDE903230A6839
:1038800004461046FFF7E0FF022814BFC2F30626E5
:103890000026002A0D46824680F2F28112F0C049CD
:1038A00040F0EE81097B002900F0EA81022803D074
:1038B0002378B34240F0E781C2F3046306931046D5
:1038C00002F07F030593FFF7C5FF059B29444FEAEC
:1038D000834848EA0A4848EA4668CE78002300222E
:1038E000CDE90823F309834648EA0008029367D02C
:1038F000059B009302466768534608A92046B847CF
:10390000002800F0C381276A4FB9414604F10C003A
:10391000FFF702FB074690B96FF0020054E03B69E5
:1039200098450DD03F68002FF9D1414604F10C00B5
:10393000FFF7F2FA07460028EED0236A3B602762C1
:1039400097F817C006F01F08CCF3840CACEB080006
:103950001FFA80FE0028B8BF0EF12000A8EB0C0370
:103960001FFA83FED7E90221B8BF00B2002B0793EC
:10397000BEBF0EF120031BB2079352EA010338D0F9
:10398000039BDFF824E39A1A049B4FF0000C63EBCF
:10399000010196457CEB01032BD36B7B97F81AE072
:1039A000734519D1029B002B78D0012821DC78685F
:1039B000F8B9DFF8F0C2944570EB010316D337E095
:1039C000276A27B96FF00C0013B0BDE8F08F3B6990
:1039D0009845B5D03F68F4E7B24890427CEB0103CC
:1039E00001D30020F0E7029B002BFAD0079B0F2B9E
:1039F00017DCFA7DB30002F0030203F07C031343EB
:103A0000FB7539462046FFF707FB6B7BBB76029BB5
:103A10003BB9FB7DC3F38402013262F38603FB757D
:103A2000D0E76A7BBB7E9A42DBD1029B002B35D06C
:103A3000B309022B32D0039BBB60049BFB601422B2
:103A400000210DA8FDF76CFF039B0A93049B0B93C9
:103A50002B1D0C932B7BADF83EB0013BDBB2ADF8D8
:103A60003C30069B8DF84230059B8DF8433094F82E
:103A70002C308DF840A083F001038DF844308DF890
:103A80004180A3680AA920469847FB7DC3F38403BD
:103A9000013303F01F039B02FB82A2E7FB7DC6F309
:103AA0004012B2EBD31F40F0F480C3F384034345CC
:103AB00040F0F280029A2B7BB609002A4DD0F20723
:103AC0005DD4032B40F2EB80039BBB60049BFB6047
:103AD0002B7BAE1D033BDBB23246394604F10C00B2
:103AE000FFF7ACFA00280CDA39462046FFF794FAC3
:103AF000FB7DC3F38403013303F01F039B02FB82AE
:103B00000AE7DDE90884AB883B834FF6FF73C9F110
:103B10002000A9F1200228FA09F104FA00F001437B
:103B200024FA02F211431846C9B2FFF7C9F909F1A4
:103B30000809B9F1400F0346E9D1B8822A7B033A5C
:103B4000D2B23146FFF7CEF9FB7DB882DA43C2F339
:103B5000C01262F3C713FB7543E786B92E1D013B04
:103B6000DBB23246394604F10C00FFF767FA002851
:103B7000BADB2A7BB88A013AD2B23146E2E7F98A47
:103B8000C1F30901013B0429DAB25BD8281D0023E7
:103B900007F11B069A4208D910F801CB06F801C0BC
:103BA000013101330529DBB2F4D103990A9104995B
:103BB0000B91934207F11B010C9138BF04337968D4
:103BC0000D9134BF55FA83F300230E93FB8AADF8B1
:103BD0003EB0C3F309031A44069B8DF84230059B9F
:103BE0008DF8433094F82C30ADF83C2083F001037D
:103BF0008DF8443000238DF840A08DF841807B6023
:103C00002A7BB88A013A291DFFF76CF93B8BB882F1
:103C1000834203D1A3680AA92046984720460AA9EF
:103C2000FFF702FEFB7DBA8AC3F38403013303F07E
:103C30001F039B02FB823B8B9A420CBF00206FF05C
:103C40001000C1E67B68002BAFD0052001E01C30DE
:103C500033461E68002EFAD1091A081D2E1D18447D
:103C600001EB090CBCF11B0F5FFA89F39DD89A4256
:103C70009BD916F8013B00F8013B09F10109EFE778
:103C80006FF00900A0E66FF00A009DE66FF00B00F0
:103C90009AE66FF00D0097E66FF00E0094E66FF075
:103CA0000F0091E640420F0080841E00EFF309836D
:103CB00005494A6B22F001024A63683383F309889D
:103CC000002383F31188704700EF00E0302080F379
:103CD000118862B60D4B0E4AD96821F4E0610904DF
:103CE000090C0A43DA60D3F8FC200A4942F08072DA
:103CF000C3F8FC20084AC2F8B01F116841F0010166
:103D000011602022DA7783F82200704700ED00E08E
:103D10000003FA0555CEACC5001000E010B5302305
:103D200083F311880E4B5B6813F4006314D0F1EE3B
:103D3000103AEFF30984683C4FF08073E361094B5C
:103D4000DB6B236684F3098800F0C4FC10B1064BDA
:103D5000A36110BD054BFBE783F31188F9E700BFB2
:103D600000ED00E000EF00E05F03000862030008E0
:103D700000F1604303F561430901C9B283F8001300
:103D8000012200F01F039A4043099B0003F16043A6
:103D900003F56143C3F880211A60704702684368E5
:103DA0001143016003B118477047000013B5446B1D
:103DB000D4F894341A681178042915D1217C022989
:103DC00012D11979128901238B4013420CD101A918
:103DD00004F14C0002F040F8D4F89444019B21799E
:103DE0000246206800F0D6F902B010BD143001F090
:103DF000C3BF00004FF0FF33143001F0BDBF00001F
:103E00004C3002F095B800004FF0FF334C3002F018
:103E10008FB80000143001F091BF00004FF0FF3167
:103E2000143001F08BBF00004C3002F061B800008C
:103E30004FF0FF324C3002F05BB8000000207047BA
:103E400010B5D0F894341A6811780429044617D1B3
:103E5000017C022914D15979528901238B401342E4
:103E60000ED1143001F024FF024648B1D4F8944436
:103E70004FF4807361792068BDE8104000F078B994
:103E800010BD0000406BFFF7DBBF00007047000073
:103E90007FB5124B036000234360C0E90233012564
:103EA00002260F4B057404460290019300F1840230
:103EB000294600964FF48073143001F0D5FE094B6B
:103EC0000294CDE9006304F523724FF48073294610
:103ED00004F14C0001F09CFF04B070BD10680008B4
:103EE000853E0008AD3D00080B68302282F3118842
:103EF0000A7903EB820210624A790D3243F82200FC
:103F00008A7912B103EB820318620223C0F8941479
:103F10000374002080F311887047000038B5037FD8
:103F2000044613B190F85430ABB9201D012502218D
:103F3000FFF734FF04F1140025776FF0010100F062
:103F400081FC84F8545004F14C006FF00101BDE88D
:103F5000384000F077BC38BD10B50121044604306C
:103F6000FFF71CFF0023237784F8543010BD0000B6
:103F700038B504460025143001F08EFE04F14C00E3
:103F8000257701F05DFF201D84F854500121FFF7D3
:103F900005FF2046BDE83840FFF752BF90F85C307F
:103FA00003F06003202B07D190F85D20212A4FF009
:103FB000000303D81F2A06D800207047222AFBD10D
:103FC000C0E9143303E0034A0265072242658365B2
:103FD000012070473823002037B5D0F894341A6890
:103FE0001178042904461AD1017C022917D11979C4
:103FF000128901238B40134211D100F14C05284650
:1040000001F0DEFF58B101A9284601F025FFD4F8E0
:104010009444019B21790246206800F0BBF803B06C
:1040200030BD0000F0B500EB810385B01E6A044688
:104030000D46FEB1302383F3118804EB8507301D54
:104040000821FFF7ABFEFB685B691B6806F14C00BB
:104050001BB1019001F00EFF019803A901F0FCFED5
:10406000024648B1039B2946204600F093F80023FE
:1040700083F3118805B0F0BDFB685A691268002A05
:10408000F5D01B8A013B1340F1D104F15C02EAE751
:104090000D3138B550F82140DCB1302383F311885D
:1040A000D4F894241368527903EB8203DB689B698C
:1040B0005D6845B104216018FFF770FE294604F1E0
:1040C000140001F0FFFD2046FFF7BAFE002383F342
:1040D000118838BD7047000001F060B910B50123A8
:1040E0000446282200F8243B0021FDF719FC002398
:1040F000C4E9013310BD000038B50446302383F312
:1041000011880025C0E90355C0E90555C0E90755E8
:10411000416001F053F90223237085F3118828468A
:1041200038BD000070B500EB810305465069DA60C8
:104130000E46144618B110220021FDF7F1FBA069CC
:1041400018B110220021FDF7EBFB31462846BDE8EF
:10415000704001F0FDB90000826802F00112826037
:104160000022C0E90422C0E90622026201F07CBA02
:10417000F0B400EB81044789E4680125A4698D400F
:104180003D43458123600023A2606360F0BC01F0E1
:1041900097BA0000F0B400EB81040789E4680125B8
:1041A00064698D403D43058123600023A260636004
:1041B000F0BC01F011BB000070B5022300250446DD
:1041C0000370C0E90255C0E90455C0E906554566CB
:1041D000056280F84C5001F057F963681B6823B101
:1041E00029462046BDE87040184770BD0378052B6E
:1041F00010B504460AD080F8683005230370436880
:104200001B680BB1042198470023A36010BD000078
:104210000178052906D190F86820436802701B6870
:1042200003B118477047000070B590F84C30044651
:1042300013B1002380F84C3004F15C02204601F0F9
:1042400035FA63689B68B3B994F85C3013F0600585
:1042500035D00021204601F0E9FC0021204601F084
:10426000DBFC63681B6813B10621204698470623D0
:1042700084F84C3070BD204698470028E4D0B4F84C
:104280006230626D9A4288BF636594F95C30656DF7
:10429000002B4FF0300380F20381002D00F0F280FC
:1042A000092284F84C2083F311880021D4E91423D7
:1042B0002046FFF76FFF002383F31188DAE794F8B5
:1042C0005D2003F07F0343EA022340F2023293426F
:1042D00000F0C58021D8B3F5807F48D00DD8012BE0
:1042E0003FD0022B00F09380002BB2D104F1640286
:1042F000226502226265A365C1E7B3F5817F00F004
:104300009B80B3F5407FA4D194F85E30012BA0D1FF
:10431000B4F8643043F0020332E0B3F5006F4DD0DF
:1043200017D8B3F5A06F31D0A3F5C063012B90D897
:10433000636894F85E205E6894F85F10B4F86030AB
:104340002046B047002884D043682365036863652E
:104350001AE0B3F5106F36D040F6024293427FF474
:1043600078AF5C4B2365022363650023C3E794F8B1
:104370005E30012B7FF46DAFB4F8643023F002039C
:10438000C4E91455A4F86430A56578E7B4F85C3046
:10439000B3F5A06F0ED194F85E3084F866302046F5
:1043A00001F0CAF863681B6813B1012120469847E1
:1043B000032323700023C4E914339CE704F167034B
:1043C00023650123C3E72378042B10D1302383F323
:1043D00011882046FFF7C0FE85F31188032163682A
:1043E00084F8675021701B680BB12046984794F8F9
:1043F0005E30002BDED084F86730042323706368BE
:104400001B68002BD6D0022120469847D2E794F8AB
:1044100060301D0603F00F0120460AD501F038F97F
:10442000012804D002287FF414AF2B4B9AE72B4BC2
:1044300098E701F01FF9F3E794F85E30002B7FF462
:1044400008AF94F8603013F00F01B3D01A0620467D
:1044500002D501F0FFFBADE701F0F2FBAAE794F80B
:104460005E30002B7FF4F5AE94F8603013F00F014E
:10447000A0D01B06204602D501F0D8FB9AE701F038
:10448000CBFB97E7142284F84C2083F311882B464A
:104490002A4629462046FFF76BFE85F31188E9E698
:1044A0005DB1152284F84C2083F311880021D4E9F2
:1044B00014232046FFF75CFEFDE60B2284F84C2017
:1044C00083F311882B462A4629462046FFF762FED1
:1044D000E3E700BF40680008386800083C6800084F
:1044E00038B590F84C300446002B3ED0063BDAB28B
:1044F0000F2A34D80F2B32D8DFE803F037313108D8
:10450000223231313131313131313737456DB0F807
:1045100062309D4214D2C3681B8AB5FBF3F203FBE1
:1045200012556DB9302383F311882B462A4629464C
:10453000FFF730FE85F311880A2384F84C300EE033
:10454000142384F84C30302383F3118800231A4657
:1045500019462046FFF70CFE002383F3118838BD6F
:10456000836D03B198470023E7E70021204601F05F
:104570005DFB0021204601F04FFB63681B6813B10F
:104580000621204698470623D7E7000010B590F88B
:104590004C30142B044629D017D8062B05D001D84F
:1045A0001BB110BD093B022BFBD80021204601F0B6
:1045B0003DFB0021204601F02FFB63681B6813B10F
:1045C000062120469847062319E0152BE9D10B2335
:1045D00080F84C30302383F3118800231A461946A3
:1045E000FFF7D8FD002383F31188DAE7C3689B69DE
:1045F0005B68002BD5D1836D03B19847002384F805
:104600004C30CEE700230375826803691B68996804
:104610009142FBD25A680360426010605860704754
:1046200000230375826803691B6899689142FBD86F
:104630005A680360426010605860704708B50846C9
:10464000302383F311880B7D032B05D0042B0DD071
:104650002BB983F3118808BD8B6900221A604FF0D3
:10466000FF338361FFF7CEFF0023F2E7D1E9003289
:1046700013605A60F3E70000FFF7C4BF054BD96829
:104680000875186802681A60536001220275D860C4
:10469000FBF750BE904B002030B50C4BDD684B1C37
:1046A00087B004460FD02B46094A684600F05EF9F1
:1046B0002046FFF7E3FF009B13B1684600F060F966
:1046C000A86907B030BDFFF7D9FFF9E7904B00208C
:1046D0003D460008044B1A68DB6890689B68984266
:1046E00094BF002001207047904B0020084B10B56C
:1046F0001C68D86822681A60536001222275DC6049
:10470000FFF78EFF01462046BDE81040FBF712BEC2
:10471000904B002038B5074C074908480123002575
:104720002370656001F084FC0223237085F31188F7
:1047300038BD00BFF84D002048680008904B0020AD
:1047400008B572B6044B186500F038FC00F01AFD8D
:10475000024B03221A70FEE7904B0020F84D002018
:1047600000F044B9034A516853685B1A9842FBD879
:10477000704700BF001000E08B60022308618B824D
:10478000084670478368A3F1840243F8142C026939
:1047900043F8442C426943F8402C094A43F8242C3E
:1047A000C26843F8182C022203F80C2C002203F8EC
:1047B0000B2C044A43F8102CA3F12000704700BFD3
:1047C0004D030008904B002008B5FFF7DBFFBDE864
:1047D0000840FFF751BF0000024BDB6898610F20D3
:1047E000FFF74CBF904B0020302383F31188FFF775
:1047F000F3BF000008B50146302383F31188082079
:10480000FFF74AFF002383F3118808BD064BDB68DE
:1048100039B1426818605A60136043600420FFF7A2
:104820003BBF4FF0FF307047904B00200368984229
:1048300006D01A680260506099611846FFF71CBFE5
:104840007047000038B504460D462068844200D108
:1048500038BD036823605C608561FFF70DFFF4E7F6
:1048600010B503689C68A2420CD85C688A600B6033
:104870004C602160596099688A1A9A604FF0FF3342
:10488000836010BD1B68121BECE700000A2938BFCB
:104890000A2170B504460D460A26601901F0C2FBD4
:1048A00001F0AEFB041BA54203D8751C2E4604463E
:1048B000F3E70A2E04D9BDE87040012001F0F8BBEF
:1048C00070BD0000F8B5144B0D46D96103F110011D
:1048D00041600A2A1969826038BF0A220160486073
:1048E0001861A818144601F08FFB0A2701F088FB15
:1048F000431BA342064606D37C1C281901F092FBF9
:1049000027463546F2E70A2F04D9BDE8F8400120D2
:1049100001F0CEBBF8BD00BF904B0020F8B50646B5
:104920000D4601F06DFB0F4A134653F8107F9F426E
:1049300006D12A4601463046BDE8F840FFF7C2BF1F
:10494000D169BB68441A2C1928BF2C46A34202D94E
:104950002946FFF79BFF224631460348BDE8F84051
:10496000FFF77EBF904B0020A04B002010B4C0E9A1
:10497000032300235DF8044B4361FFF7CFBF000022
:1049800010B5194C236998420DD0D0E900328168E6
:1049900013605A609A680A449A60002303604FF0DB
:1049A000FF33A36110BD2346026843F8102F536004
:1049B0000022026022699A4203D1BDE8104001F052
:1049C0002BBB936881680B44936001F019FB22694B
:1049D000E1699268441AA242E4D91144BDE810404A
:1049E000091AFFF753BF00BF904B00202DE9F04795
:1049F000DFF8BC8008F110072C4ED8F8105001F0F9
:104A0000FFFAD8F81C40AA68031B9A423ED8144407
:104A1000D5E900324FF00009C8F81C4013605A6015
:104A2000C5F80090D8F81030B34201D101F0F4FA83
:104A300089F31188D5E9033128469847302383F359
:104A400011886B69002BD8D001F0DAFA6A69A0EB03
:104A500004094A4582460DD2022001F029FB0022BA
:104A6000D8F81030B34208D151462846BDE8F04787
:104A7000FFF728BF121A2244F2E712EB090938BFE8
:104A80004A4629463846FFF7EBFEB5E7D8F810301E
:104A9000B34208D01444211AC8F81C00A960BDE82C
:104AA000F047FFF7F3BEBDE8F08700BFA04B002042
:104AB000904B002038B501F0A3FA054AD2E9084529
:104AC000031B181945F10001C2E9080138BD00BFF8
:104AD000904B002000207047FEE700007047000068
:104AE0004FF0FF307047000002290CD0032904D09A
:104AF0000129074818BF00207047032A05D8054838
:104B000000EBC2007047044870470020704700BFA8
:104B10002069000848230020D468000870B59AB0C6
:104B20000546084601A9144600F0C2F801A8FCF7A2
:104B3000EFFE431C5B00C5E9003400222370032311
:104B40006370C6B201AB02341046D1B28E4204F19A
:104B5000020401D81AB070BD13F8011B04F8021C3E
:104B600004F8010C0132F0E708B5302383F3118813
:104B70000348FFF731FA002383F3118808BD00BF13
:104B8000004E002090F85C3003F01F02012A07D18C
:104B900090F85D200B2A03D10023C0E9143315E0FF
:104BA00003F06003202B08D1B0F860302BB990F8E7
:104BB0005D20212A03D81F2A04D8FFF7EFB9222A43
:104BC000EBD0FAE7034A02650722426583650120BC
:104BD000704700BF3F23002007B5052917D8DFE83D
:104BE00001F0191603191920302383F31188104A94
:104BF00001900121FFF796FA01980E4A0221FFF772
:104C000091FA0D48FFF7B4F9002383F3118803B03C
:104C10005DF804FB302383F311880748FFF77EF922
:104C2000F2E7302383F311880348FFF795F9EBE7A8
:104C30007468000898680008004E002038B50C4DD4
:104C40000C4C0D492A4604F10800FFF767FF05F1F7
:104C5000CA0204F110000949FFF760FF05F5CA72A6
:104C600004F118000649BDE83840FFF757BF00BF00
:104C7000C852002048230020546800085E680008DD
:104C80006968000870B5044608460D46FCF740FE0A
:104C9000C6B22046013403780BB9184670BD3246BF
:104CA0002946FCF721FE0028F3D10120F6E7000099
:104CB0002DE9F84F05460C46FCF72AFE2B49C6B2F3
:104CC0002846FFF7DFFF08B10336F6B22849284629
:104CD000FFF7D8FF08B11036F6B2632E0DD8DFF813
:104CE0008C80DFF88C90234FDFF890A0DFF890B035
:104CF0002E7846B92670BDE8F88F29462046BDE8D3
:104D0000F84F01F01BBD252E2BD107224146284626
:104D1000FCF7EAFD58B9DBF800302360DBF804301B
:104D20006360BBF80830238107350A34E0E70822C6
:104D300049462846FCF7D8FD98B90F4BA21C1978B4
:104D400009090232C95D02F8041C13F8011B01F0C5
:104D50000F015345C95D02F8031CF0D11834083522
:104D6000C6E704F8016B0135C2E700BF40690008DF
:104D70006968000848690008107AF01F1C7AF01F63
:104D80005A670008BFF34F8F024AD368DB03FCD495
:104D9000704700BF003C024008B5074B1B7853B971
:104DA000FFF7F0FF054B1A69002ABFBF044A5A609B
:104DB00002F188325A6008BD26550020003C0240AE
:104DC0002301674508B5054B1B7833B9FFF7DAFFB8
:104DD000034A136943F00043136108BD26550020C0
:104DE000003C02400728F0B516D80C4C0C4923783B
:104DF0007BB90C4D0E4608234FF0006255F8047B3A
:104E000046F8042B013B13F0FF033A44F6D101238B
:104E1000237051F82000F0BD0020FCE74855002029
:104E2000285500205C690008014B53F820007047AA
:104E30005C69000808207047072810B5044601D9AE
:104E4000002010BDFFF7CEFF064B53F82430184466
:104E5000C21A0BB90120F4E712680132F0D1043B09
:104E6000F6E700BF5C690008072810B5044621D8A2
:104E7000FFF788FFFFF790FF0F4AF323D360C300CB
:104E8000DBB243F4007343F002031361136943F48C
:104E900080331361FFF776FFFFF7A4FF074B53F84A
:104EA000241000F04BF9FFF78DFF2046BDE81040BD
:104EB000FFF7C2BF002010BD003C02405C69000843
:104EC000F8B512F00103144642D185182E4A9542D6
:104ED00057D82E4B1B6813F0010352D02C4DFFF70F
:104EE0005BFFF323EB60FFF74DFF40F20127032C3C
:104EF00015D824F001046618254C401A40F2011719
:104F0000B142236900EB010524D123F001032361A1
:104F1000FFF758FF0120F8BD043C0430E7E78307A2
:104F2000E7D12B6923F440732B612B693B432B6141
:104F300051F8046B0660BFF34F8FFFF723FF036840
:104F40009E42E9D02B6923F001032B61FFF73AFF62
:104F50000020E0E723F44073236123693B4323618E
:104F60000B882B80BFF34F8FFFF70CFF2D8831F894
:104F7000023BADB2AB42C3D0236923F001032361EE
:104F8000E4E71846C7E700BF000008080038024001
:104F9000003C0240084908B50B7828B11BB9FFF75F
:104FA000FBFE01230B7008BD002BFCD0BDE80840C0
:104FB0000870FFF707BF00BF2655002008B50B4853
:104FC0004FF47F4100F0CCF809484FF4303100F045
:104FD000C7F808484FF4804100F0C2F8BDE8084027
:104FE0004FF470514FF4805000F0BAB80001002027
:104FF0000000012000C003200846114601F002BB5A
:10500000012001F0FFBA0000084601F019BB0000C2
:1050100038B5EFF311859DB9EFF30584C4F30804A7
:10502000302334B183F31188FFF744FD85F31188F1
:1050300038BD83F31188FFF73DFD84F3118838BD37
:10504000BDE83840FFF736BD38B5FFF7E1FF114C3A
:10505000114AC00840EA4170A0FB025EC908A0FBEB
:10506000040C1CEB050CA1FB04404FF000035B415A
:10507000A1FB02121CEB040C43EB000011EB0E0130
:1050800042F10002411842F10000090941EA0070B2
:1050900038BD00BFCFF753E3A59BC42010B5024431
:1050A000064BD2B2904200D110BD441C00B253F85E
:1050B000200041F8040BE0B2F4E700BF50280040A4
:1050C0000F4B30B51C6F240407D41C6F44F40074DC
:1050D0001C671C6F44F400441C670A4C236843F4AB
:1050E000807323600244084BD2B2904200D130BD9D
:1050F000441C00B251F8045B43F82050E0B2F4E7DE
:1051000000380240007000405028004007B50122DE
:1051100001A90020FFF7C2FF019803B05DF804FB6E
:1051200013B50446FFF7F2FFA04205D0012201A902
:1051300000200194FFF7C4FF02B010BD0144BFF38B
:105140004F8F064B884204D3BFF34F8FBFF36F8F4F
:105150007047C3F85C022030F4E700BF00ED00E0C8
:105160000144BFF34F8F064B884204D3BFF34F8FE8
:10517000BFF36F8F7047C3F870022030F4E700BFB1
:1051800000ED00E070470000074B45F255521A60F1
:1051900002225A6040F6FF729A604CF6CC421A60C6
:1051A000024B01221A707047003000405055002019
:1051B000034B1B781BB1034B4AF6AA221A607047B7
:1051C0005055002000300040034B1A681AB9034ABA
:1051D000D2F874281A6070474C5500200030024005
:1051E000024B4FF08072C3F87428704700300240C1
:1051F00008B5FFF7E9FF024B1868C0F3407008BD1F
:105200004C55002008B5FFF7DFFF024B1868C0F3CC
:10521000007008BD4C55002070B5BFF34F8FBFF331
:105220006F8F1A4A0021C2F85012BFF34F8FBFF39D
:105230006F8F536943F400335361BFF34F8FBFF354
:105240006F8FC2F88410BFF34F8FD2F88030C3F352
:10525000C900C3F34E335B0143F6E07403EA04066E
:10526000014646EA81750139C2F86052F9D2203B05
:1052700013F1200FF2D1BFF34F8F536943F4803302
:105280005361BFF34F8FBFF36F8F70BD00ED00E030
:10529000FEE7000070B5214B2148224A904237D3E7
:1052A000214BDA1C121AC11E22F003028B4238BFB6
:1052B00000220021FCF734FB1C4A0023C2F8843092
:1052C000BFF34F8FD2F88030C3F3C900C3F34E331E
:1052D0005B0143F6E07403EA0406014646EA817581
:1052E0000139C2F86C52F9D2203B13F1200FF2D1F0
:1052F000BFF34F8FBFF36F8FBFF34F8FBFF36F8F2E
:105300000023C2F85032BFF34F8FBFF36F8F70BDD1
:1053100053F8041B40F8041BC0E700BF846B00086F
:105320006C5600206C5600206C56002000ED00E00A
:1053300070B5D0E91B439E6800224FF0FF3504EBA7
:1053400042135101D3F800090028BEBFD3F8000969
:1053500040F08040C3F80009D3F8000B0028BEBF1E
:10536000D3F8000B40F08040C3F8000B0132631803
:105370009642C3F80859C3F8085BE0D24FF0011316
:10538000C4F81C3870BD0000890141F020010161A2
:1053900003699B06FCD41220FFF7E4B910B5054C55
:1053A0002046FEF79BFE4FF0A043E366024B2367C7
:1053B00010BD00BF54550020A069000870B50378E7
:1053C000012B054650D12A4BC46E98421BD1294B64
:1053D0005A6B42F080025A635A6D42F080025A655D
:1053E0005A6D5A6942F080025A615A6922F080026D
:1053F0005A610E2143205B69FEF7BAFC1E4BE36045
:105400001E4BC4F800380023C4F8003EC0232360BC
:10541000EE6E4FF40413A3633369002BFCDA01230F
:1054200033610C20FFF79EF93369DB07FCD41220AF
:10543000FFF798F93369002BFCDA0026A6602846AE
:10544000FFF776FF6B68C4F81068DB68C4F814686F
:10545000C4F81C684BB90A4BA3614FF0FF3363617A
:10546000A36843F00103A36070BD064BF4E700BFDF
:105470005455002000380240401400400300200230
:10548000003C30C0083C30C0F8B5C46E0546002171
:105490002046FFF779FF296F00234FF001128F6834
:1054A000C4F834384FF00066C4F81C284FF0FF30C1
:1054B00004EB431201339F42C2F80069C2F8006B4B
:1054C000C2F80809C2F8080BF2D20B68EA6E6B67E3
:1054D000636210231361166916F01006FBD11220C7
:1054E000FFF740F9D4F8003823F4FE63C4F800381D
:1054F000A36943F4402343F01003A3610923C4F8D4
:105500001038C4F814380A4BEB604FF0C043C4F8AD
:10551000103B084BC4F8003BC4F81069C4F80039CC
:105520006B6F03F1100243F480136A67A362F8BD46
:105530007C69000840800010C26E90F86610D2F8B6
:10554000003823F4FE6343EA0113C2F800387047C1
:105550002DE9F84300EB8103C56EDA68166806F0A2
:105560000306731E022B05EB41130C4680460FFA0F
:1055700081F94FEA41104FF00001C3F8101B4FF0C2
:10558000010104F1100398BFB60401FA03F3916915
:105590008EBF334E06F1805606F5004600293AD0FC
:1055A000578A04F15801490137436F50D5F81C1848
:1055B0000B43C5F81C382B180021C3F81019536988
:1055C0000127611EA7409BB3138A928B9B08012A77
:1055D00088BF5343D8F87420981842EA034301F176
:1055E000400205EB8202C8F8740021465360284649
:1055F000FFF7CAFE08EB8900C3681B8A43EA84539D
:10560000483464011E432E51D5F81C381F43C5F899
:105610001C78BDE8F88305EB4917D7F8001B21F487
:105620000041C7F8001BD5F81C1821EA0303C0E7A6
:1056300004F13F0305EB83030A4A5A6028462146DA
:10564000FFF7A2FE05EB4910D0F8003923F4004320
:10565000C0F80039D5F81C3823EA0707D7E700BFA0
:105660000080001000040002026F12684267FFF71A
:105670005FBE00005831C36E49015B5813F400400F
:1056800004D013F4001F0CBF02200120704700005B
:105690004831C36E49015B5813F4004004D013F441
:1056A000001F0CBF022001207047000000EB8101A9
:1056B000CB68196A0B6813604B6853607047000031
:1056C00000EB810330B5DD68AA691368D36019B9AE
:1056D000402B84BF402313606B8A1468C26E1C4445
:1056E000013CB4FBF3F46343033323F0030302EB05
:1056F000411043EAC44343F0C043C0F8103B2B6859
:1057000003F00303012B09B20ED1D2F8083802EBE3
:10571000411013F4807FD0F8003B14BF43F0805356
:1057200043F00053C0F8003B02EB4112D2F8003BBB
:1057300043F00443C2F8003B30BD00002DE9F041C6
:10574000244DEE6E06EB40130446D3F8087BC3F8F5
:10575000087B38070AD5D6F81438190706D505EBA3
:1057600084032146DB6828465B689847FA071FD503
:10577000D6F81438DB071BD505EB8403D968CCB900
:105780008B69488A5A68B2FBF0F600FB16228AB988
:105790001868DA6890420DD2121AC3E90024302347
:1057A00083F311880B482146FFF78AFF84F31188A1
:1057B000BDE8F081012303FA04F26B8923EA0203B6
:1057C0006B81CB68002BF3D021460248BDE8F04145
:1057D000184700BF5455002000EB810370B5DD6809
:1057E000C36E6C692668E6604A0156BB1A444FF4E2
:1057F0000020C2F810092A6802F00302012A0AB246
:105800000ED1D3F8080803EB421410F4807FD4F8CB
:10581000000914BF40F0805040F00050C4F8000967
:1058200003EB4212D2F8000940F00440C2F800092C
:10583000D3F83408012202FA01F10143C3F8341805
:1058400070BD19B9402E84BF4020206020682E8A88
:105850008419013CB4FBF6F440EAC44040F0005027
:105860001A44C6E72DE9F8433B4DEE6E06EB4013B4
:105870000446D3F80889C3F8088918F0010F4FEAE5
:1058800040171AD0D6F81038DB0716D505EB800381
:10589000D9684B691868DA68904230D2121A4FF012
:1058A00000091A60C3F80490302383F3118821465D
:1058B0002846FFF791FF89F3118818F0800F1CD05C
:1058C000D6F834380126A640334216D005EB8403BF
:1058D000ED6ED3F80CC0DCF814200134E4B2D2F839
:1058E00000E005EB04342F445168714515D3D5F819
:1058F000343823EA0606C5F83468BDE8F883012386
:1059000003FA04F22B8923EA02032B818B68002B14
:10591000D3D0214628469847CFE7BCF81000AEEB1D
:105920000103834228BF0346D7F8180980B2B3EBBE
:10593000800FE2D89068A0F1040959F8048FC4F8E8
:105940000080A0EB09089844B8F1040FF5D818447A
:105950000B4490605360C7E7545500202DE9F74F82
:10596000AC4CE56E6E69AB691E4016F480586E61F2
:1059700007D02046FEF720FC03B0BDE8F04FFEF74D
:10598000CDB9002E12DAD5F8003EA2489B071EBF03
:10599000D5F8003E23F00303C5F8003ED5F80438DF
:1059A00023F00103C5F80438FEF732FC370505D5AE
:1059B0009848FFF7BDFC9748FEF718FCB0040CD5DB
:1059C000D5F8083813F0060FEB6823F470530CBFBA
:1059D00043F4105343F4A053EB6031071BD56368C5
:1059E000DB681BB9AB6923F00803AB612378052B97
:1059F0000CD1D5F8003E87489A071EBFD5F8003E67
:105A000023F00303C5F8003EFEF702FC6368DB6881
:105A10000BB180489847F30200F18980B70227D57F
:105A2000D4F86C90DFF8ECB100274FF0010A09EBD5
:105A30004712D2F8003B03F44023B3F5802F11D175
:105A4000D2F8003B002B0DDA62890AFA07F322EA4A
:105A50000303638104EB8703DB68DB6813B139461A
:105A600058469847236F01379B68FFB29F42DED9A3
:105A7000F00617D5E76E3A6AC2F30A1002F00F0378
:105A800002F4F012B2F5802F00F09980B2F5402FA9
:105A900008D104EB83030022DB681B6A07F58057FB
:105AA00090427ED13303D5F818481DD5E70302D5BF
:105AB0000020FFF743FEA50302D50120FFF73EFEBD
:105AC000600302D50220FFF739FE210302D503202F
:105AD000FFF734FEE20202D50420FFF72FFEA302F7
:105AE00002D50520FFF72AFE77037FF545AFE607CD
:105AF00002D50020FFF7B6FEA50702D50120FFF76B
:105B0000B1FE600702D50220FFF7ACFE210702D5E7
:105B10000320FFF7A7FEE20602D50420FFF7A2FE4E
:105B2000A3067FF529AF0520FFF79CFE24E7E36E6F
:105B3000DFF8E0A0019300274FF00109236F9B6875
:105B40005FFA87FB9B453FF669AF019B03EB4B1365
:105B5000D3F8001901F44021B1F5802F1FD1D3F8FB
:105B6000001900291BDAD3F8001941F09041C3F85D
:105B70000019D3F800190029FBDB5946E06EFFF746
:105B800003FC218909FA0BF321EA0303238104EBC7
:105B90008B03DB689B6813B1594650469847013721
:105BA000CCE7910708BFD7F80080072A98BF03F811
:105BB000018B02F1010298BF4FEA182870E7023307
:105BC00004EB830207F580575268D2F818C0DCF85E
:105BD0000820DCE9001CA1EB0C0C002188420AD152
:105BE00004EB830463689B699A6802449A605A686C
:105BF00002445A6056E711F0030F08BFD7F800803F
:105C00008C4588BF02F8018B01F1010188BF4FEA82
:105C10001828E3E754550020C36E03EB4111D1F877
:105C2000003B43F40013C1F8003B7047C36E03EB25
:105C30004111D1F8003943F40013C1F8003970471D
:105C4000C36E03EB4111D1F8003B23F40013C1F8FC
:105C5000003B7047C36E03EB4111D1F8003923F4C8
:105C60000013C1F80039704730B5039C017204334A
:105C700004FB0325C0E90653049B03630021059B35
:105C8000C160C0E90000C0E90422C0E90842C0E9DF
:105C90000A11436330BD0000416A0022C0E90411CB
:105CA000C0E90A22C2606FF00101FEF7CBBD00001F
:105CB000D0E90432934201D1C2680AB9181D704775
:105CC0000020704703691960C2680132C260C2696E
:105CD000134482690361934224BF436A0361002134
:105CE000FEF7A4BD38B504460D46E3683BB16269D2
:105CF000131D1268A3621344E362002007E0237AB5
:105D000033B929462046FEF781FD0028EDDA38BD7B
:105D10006FF00100FBE70000C368C269013BC3608C
:105D20004369134482694361934224BF436A4361D8
:105D300000238362036B03B11847704770B53023AB
:105D4000044683F31188866A3EB9FFF7CBFF054608
:105D500018B186F31188284670BDA36AE26A13F869
:105D6000015BA362934202D32046FFF7D5FF0023D5
:105D700083F31188EFE700002DE9F84F04460E4643
:105D8000174698464FF0300989F311880025AA4636
:105D9000D4F828B0BBF1000F09D141462046FFF7E7
:105DA000A1FF20B18BF311882846BDE8F88FD4E914
:105DB0000A12A7EB050B521A934528BF9346BBF175
:105DC000400F1BD9334601F1400251F8040B43F850
:105DD000040B9142F9D1A36A40334036A3624035A7
:105DE000D4E90A239A4202D32046FFF795FF8AF3AB
:105DF0001188BD42D8D289F31188C9E730465A4686
:105E0000FBF768FDA36A5B445E44A3625D44E7E779
:105E100010B5029C0172043303FB0421C0E9061390
:105E20000023C0E90A33039B0363049BC460C0E9F9
:105E30000000C0E90422C0E90842436310BD00002D
:105E4000026AC260426AC0E904220022C0E90A2252
:105E50006FF00101FEF7F6BCD0E904239A4201D1AC
:105E6000C26822B9184650F8043B0B607047002303
:105E70001846FAE7C368C2690133C3604369134433
:105E800082694361934224BF436A43610021FEF764
:105E9000CDBC000038B504460D46E3683BB123692C
:105EA0001A1DA262E2691344E362002007E0237A2C
:105EB00033B929462046FEF7A9FC0028EDDA38BDA3
:105EC0006FF00100FBE7000003691960C268013A46
:105ED000C260C269134482690361934224BF436A6A
:105EE000036100238362036B03B11847704700000E
:105EF00070B530230D460446114683F31188866A37
:105F00002EB9FFF7C7FF10B186F3118870BDA36AE1
:105F10001D70A36AE26A01339342A36204D3E1696C
:105F200020460439FFF7D0FF002080F31188EDE709
:105F30002DE9F84F04460D46904699464FF0300A39
:105F40008AF311880026B346A76A4FB9494620460E
:105F5000FFF7A0FF20B187F311883046BDE8F88F26
:105F6000D4E90A073A1AA8EB0607974228BF174652
:105F7000402F1BD905F1400355F8042B40F8042BA2
:105F80009D42F9D1A36A4033A3624036D4E90A2383
:105F90009A4204D3E16920460439FFF795FF8BF359
:105FA00011884645D9D28AF31188CDE729463A4669
:105FB000FBF790FCA36A3B443D44A3623E44E5E703
:105FC000D0E904239A4217D1C3689BB1836A8BB18D
:105FD000043B9B1A0ED01360C368013BC360C369C6
:105FE0001A44836902619A4224BF436A0361002311
:105FF00083620123184670470023FBE700F0D2B804
:106000004FF08043586A70474FF080430022586336
:106010001A610222DA6070474FF080430022DA6092
:10602000704700004FF0804358637047FEE7000060
:1060300070B51B4B01630025044686B0586085622D
:106040000E46FDF743FE04F11003C4E904334FF09C
:10605000FF33C4E90635C4E90044A560E562FFF7F3
:10606000CFFF2B460246C4E9082304F134010D4A50
:10607000256580232046FEF77FFB0123E0600A4A66
:106080000375009272680192B268CDE90223074B52
:106090006846CDE90435FEF797FB06B070BD00BF3A
:1060A000F84D0020AC690008B16900082D600008B7
:1060B000024AD36A1843D062704700BF904B002059
:1060C0004B6843608B688360CB68C3600B69436136
:1060D0004B6903628B6943620B6803607047000081
:1060E00008B5264B26481A6940F2FF110A431A6187
:1060F0001A6922F4FF7222F001021A611A691A6BFE
:106100000A431A631A6D0A431A651E4A1B6D11462B
:10611000FFF7D6FF02F11C0100F58060FFF7D0FF0A
:1061200002F1380100F58060FFF7CAFF02F1540167
:1061300000F58060FFF7C4FF02F1700100F5806098
:10614000FFF7BEFF02F18C0100F58060FFF7B8FF9A
:1061500002F1A80100F58060FFF7B2FF02F1C4016F
:1061600000F58060FFF7ACFF02F1E00100F5806010
:10617000FFF7A6FFBDE8084000F088B800380240ED
:1061800000000240B869000808B500F0F3F9FEF716
:10619000C1FAFFF719F8BDE80840FEF74FBD00004F
:1061A000704700000F4B1A6C42F001021A641A6E1D
:1061B00042F001021A660C4A1B6E936843F0010319
:1061C00093604FF080436B229A624FF0FF32DA62A5
:1061D00000229A615A63DA605A6001225A611A6099
:1061E000704700BF00380240002004E04FF08042BA
:1061F00008B51169D3680B40D9B2C9439B07116137
:1062000007D5302383F31188FEF7AAFA002383F31E
:10621000118808BD1B4B1A696FEAC2526FEAD2524D
:106220001A611A69C2F308021A614FF0FF301A6945
:106230005A69586100215A6959615A691A6A62F0AB
:1062400080521A621A6A02F080521A621A6A5A6AF4
:1062500058625A6A59625A6A0B4A106840F4807050
:106260001060186F00F44070B0F5007F1EBF4FF44F
:10627000803018671967536823F40073536000F087
:1062800055B900BF0038024000700040364B374A15
:106290001A64374A4FF4404111601A6842F0010213
:1062A0001A601A689207FCD59A6822F003029A6075
:1062B0002D4B9A6812F00C02FBD1196801F0F9011C
:1062C00019609A601A6842F480321A601A68900362
:1062D000FCD55A6F42F001025A67234B5A6F91075F
:1062E000FCD5244A5A601A6842F080721A60204B2A
:1062F0005A685204FCD51A6842F480321A605A680F
:10630000D003FCD51A6842F400321A60184A536868
:106310009903FCD5144B1A689201FCD5164A9A6071
:1063200040F20112C3F88C200022C3F89020134AD7
:1063300040F207331360136803F00F03072BFAD101
:10634000094B9A6842F002029A609A6802F00C02C5
:10635000082AFAD15A6C42F480425A645A6E42F4C6
:1063600080425A665B6E704700380240000400109D
:1063700000700040106C400900948838003C0240D6
:10638000074A08B5536903F00103536123B1054A75
:1063900013680BB150689847BDE80840FDF7BEBCD4
:1063A000003C0140E4550020074A08B5536903F05A
:1063B0000203536123B1054A93680BB1D068984733
:1063C000BDE80840FDF7AABC003C0140E4550020B0
:1063D000074A08B5536903F00403536123B1054A22
:1063E00013690BB150699847BDE80840FDF796BCAA
:1063F000003C0140E4550020074A08B5536903F00A
:106400000803536123B1054A93690BB1D0699847DA
:10641000BDE80840FDF782BC003C0140E455002087
:10642000074A08B5536903F01003536123B1054AC5
:10643000136A0BB1506A9847BDE80840FDF76EBC7F
:10644000003C0140E4550020164B10B55C6904F493
:1064500078725A61A30604D5134A936A0BB1D06AC5
:106460009847600604D5104A136B0BB1506B9847E0
:10647000210604D50C4A936B0BB1D06B9847E2050B
:1064800004D5094A136C0BB1506C9847A30504D589
:10649000054A936C0BB1D06C9847BDE81040FDF7EE
:1064A0003DBC00BF003C0140E4550020194B10B535
:1064B0005C6904F47C425A61620504D5164A136D86
:1064C0000BB1506D9847230504D5134A936D0BB15A
:1064D000D06D9847E00404D50F4A136E0BB1506E8F
:1064E0009847A10404D50C4A936E0BB1D06E98471F
:1064F000620404D5084A136F0BB1506F9847230408
:1065000004D5054A936F0BB1D06F9847BDE8104092
:10651000FDF704BC003C0140E455002008B5FFF73E
:1065200065FEBDE80840FDF7F9BB0000062108B58F
:106530000846FDF71DFC06210720FDF719FC062182
:106540000820FDF715FC06210920FDF711FC0621A6
:106550000A20FDF70DFC06211720FDF709FC062196
:106560002820FDF705FCBDE8084007211C20FDF7A9
:10657000FFBB000008B5FFF74DFE00F00BF8FDF77C
:10658000ABFDFDF783FCFFF70BFEBDE80840FFF70E
:1065900035BD00000023054A19460133102BC2E91E
:1065A000001102F10802F8D1704700BFE455002045
:1065B0000B460146184600F02DB8000000F040B828
:1065C000012838BF012010B50446204600F030F8FD
:1065D00030B900F007F808B900F00CF88047F4E78C
:1065E00010BD0000024B1868BFF35B8F704700BFFF
:1065F0006456002008B5062000F084F80120FEF75C
:106600006BFA0000024B0A4601461868FEF7F4BC1C
:106610006823002010B5054C13462CB10A460146EC
:106620000220AFF3008010BD2046FCE70000000010
:10663000024B01461868FEF7E3BC00BF6823002048
:10664000024B01461868FEF7DFBC00BF682300203C
:1066500010B501390244904201D1002005E00378D1
:1066600011F8014FA34201D0181B10BD0130F2E711
:106670002DE9F041A3B1C91A17780144044603F18A
:10668000FF3C8C42204601D9002009E00578BD423C
:1066900004F10104F5D10CEB0405D618A54201D193
:1066A000BDE8F08115F8018D16F801EDF045F5D043
:1066B000E7E700001F2938B504460D4604D9162324
:1066C00003604FF0FF3038BD426C12B152F82130F8
:1066D0004BB9204600F030F82A4601462046BDE876
:1066E000384000F017B8012B0AD0591C03D11623EB
:1066F00003600120E7E7002442F825402846984738
:106700000020E0E7024B01461868FFF7D3BF00BF47
:106710006823002038B5074D00230446084611467B
:106720002B60FEF7DDF9431C02D12B6803B1236017
:1067300038BD00BF68560020FEF7CCB9034611F8FB
:10674000012B03F8012B002AF9D170476F72672ED5
:106750006172647570696C6F742E46726565666CE3
:106760007952544B0000000053544D3332463F3FA2
:106770003F3F3F3F0053544D333246375B347C3507
:106780005D780053544D333246375B367C375D7845
:106790000000000040A2E4F1646891060041A3E516
:1067A000F2656992070000004261642043414E494E
:1067B0006661636520696E6465782E008000000064
:1067C00000800000000080000000000000000000C9
:1067D000E5210008012A00085D290008252200089B
:1067E0003122000831240008F521000805220008A4
:1067F000F921000801220008FD21000855230008A6
:1068000009220008D12C00081922000829230008B9
:1068100000000000093E0008F53D0008313E000878
:106820001D3E0008293E0008153E0008013E0008F4
:10683000ED3D00083D3E00080000000001000000A2
:10684000000000006330000044680008E84B0020AE
:10685000F84D00204172647550696C6F74002542D8
:106860004F415244252D424C002553455249414C3D
:106870002500000002000000000000002540000884
:10688000914000084000400098520020A85200208B
:1068900002000000000000000300000000000000F3
:1068A000D54000080000000010000000B852002091
:1068B000000000000100000000000000545500200E
:1068C00001010200D94B0008E94A0008854B000885
:1068D000694B000843000000DC680008090243001F
:1068E000020100C032090400000102020100052477
:1068F0000010010524010001042402020524060001
:1069000001070582030800FF09040100020A0000D4
:106910000007050102400000070581024000000059
:106920001200000028690008120110010200004056
:106930000912415700020102030100000403090487
:1069400025424F41524425003031323334353637F9
:1069500038394142434445460000000000400000F1
:106960000040000000400000004000000000010066
:106970000000020000000200000002000000000011
:1069800029420008E14400088D450008400040000D
:10699000CC550020CC55002001000000DC55002023
:1069A0008000000040010000050000006D61696E7C
:1069B0000069646C650000000010806A000000003F
:1069C000AAAAAAAA00000064FFFF000000000000BD
:1069D00000A00A0000000A0000000000AAAAAAAA5B
:1069E00000000000FFFF0000000000009900000010
:1069F0000040000000000000AAAAAAAA000000208F
:106A0000FFFF000000000000000000000000000088
:106A100000000000AAAAAAAA00000000FFFF0000D0
:106A20000000000000000000000000000000000066
:106A3000AAAAAAAA00000000FFFF000000000000B0
:106A4000000000000000000000000000AAAAAAAA9E
:106A500000000000FFFF0000000000000000000038
:106A60000000000000000000AAAAAAAA000000007E
:106A7000FFFF000000000000000000000000000018
:106A8000000000000A0000000000000003000000F9
:106A900000000000000000000000000000000000F6
:106AA00000000000000000000000000000000000E6
:106AB00000000000000000000404000000000000CE
:106AC000000007000000000040420F00FE2A010005
:106AD000D2040000FF00000000000000686700080A
:106AE000490400007567000851040000836700082E
:106AF000009600000000080096000000000800005A
:106B0000040000003C6900080000000000000000D4
:106B10000000000000000000000000000000000075
:106B20006C230020000000000000000000000000B6
:106B30000000000000000000000000000000000055
:106B40000000000000000000000000000000000045
:106B50000000000000000000000000000000000035
:106B60000000000000000000000000000000000025
:106B70000000000000000000000000000000000015
:046B80000000000011
:00000001FF
